 EMenu

 Timestamp is 56b152ea (Wed Feb 03 04:07:54 2016)

 Preferred load address is 10000000

 Start         Length     Name                   Class
 0001:00000000 000001b0H .idata$5                CODE
 0001:000001b0 00000004H .CRT$XCA                CODE
 0001:000001b4 00000004H .CRT$XCZ                CODE
 0001:000001b8 00000004H .CRT$XIA                CODE
 0001:000001bc 0000000cH .CRT$XIC                CODE
 0001:000001c8 00000004H .CRT$XIZ                CODE
 0001:000001cc 00000004H .CRT$XPA                CODE
 0001:000001d0 00000004H .CRT$XPZ                CODE
 0001:000001d4 00000004H .CRT$XTA                CODE
 0001:000001d8 00000004H .CRT$XTZ                CODE
 0001:000001e0 000023c0H .rdata                  CODE
 0001:000025a0 000000dcH .rdata$r                CODE
 0001:00002680 00000010H .rdata$sxdata           CODE
 0001:00002690 00000004H .rtc$IAA                CODE
 0001:00002694 00000004H .rtc$IZZ                CODE
 0001:00002698 00000004H .rtc$TAA                CODE
 0001:0000269c 00000004H .rtc$TZZ                CODE
 0001:000026a0 0000e0aaH .text                   CODE
 0001:0001074a 00000014H .text$yd                CODE
 0001:00010760 0000029cH .xdata$x                CODE
 0001:000109fc 00000050H .idata$2                CODE
 0001:00010a4c 00000014H .idata$3                CODE
 0001:00010a60 000001b0H .idata$4                CODE
 0001:00010c10 0000077aH .idata$6                CODE
 0001:00011390 000000b6H .edata                  CODE
 0002:00000000 00000ed8H .data                   DATA
 0002:00000ee0 000016e0H .bss                    DATA
 0003:00000000 000000a0H .rsrc$01                DATA
 0003:000000a0 000003a0H .rsrc$02                DATA

  Address         Publics by Value              Rva+Base       Lib:Object

 0000:00000000       __except_list              00000000     <absolute>
 0000:00000004       ___safe_se_handler_count   00000004     <absolute>
 0000:00000000       ___ImageBase               10000000     <linker-defined>
 0001:00000000       __imp__lstrcpynW@12        10001000     kernel32:KERNEL32.dll
 0001:00000004       __imp__lstrcatW@8          10001004     kernel32:KERNEL32.dll
 0001:00000008       __imp__lstrlenW@4          10001008     kernel32:KERNEL32.dll
 0001:0000000c       __imp__lstrcmpW@8          1000100c     kernel32:KERNEL32.dll
 0001:00000010       __imp__CompareStringW@24   10001010     kernel32:KERNEL32.dll
 0001:00000014       __imp__lstrcpyW@8          10001014     kernel32:KERNEL32.dll
 0001:00000018       __imp__MultiByteToWideChar@24 10001018     kernel32:KERNEL32.dll
 0001:0000001c       __imp__lstrlenA@4          1000101c     kernel32:KERNEL32.dll
 0001:00000020       __imp__CloseHandle@4       10001020     kernel32:KERNEL32.dll
 0001:00000024       __imp__SetEvent@4          10001024     kernel32:KERNEL32.dll
 0001:00000028       __imp__WaitForMultipleObjects@16 10001028     kernel32:KERNEL32.dll
 0001:0000002c       __imp__CreateThread@24     1000102c     kernel32:KERNEL32.dll
 0001:00000030       __imp__GetExitCodeThread@8 10001030     kernel32:KERNEL32.dll
 0001:00000034       __imp__CreateEventW@16     10001034     kernel32:KERNEL32.dll
 0001:00000038       __imp__WaitForSingleObject@8 10001038     kernel32:KERNEL32.dll
 0001:0000003c       __imp__TerminateThread@8   1000103c     kernel32:KERNEL32.dll
 0001:00000040       __imp__VerifyVersionInfoW@16 10001040     kernel32:KERNEL32.dll
 0001:00000044       __imp__VerSetConditionMask@16 10001044     kernel32:KERNEL32.dll
 0001:00000048       __imp__GetModuleHandleW@4  10001048     kernel32:KERNEL32.dll
 0001:0000004c       __imp__GetFileAttributesW@4 1000104c     kernel32:KERNEL32.dll
 0001:00000050       __imp__lstrcmpA@8          10001050     kernel32:KERNEL32.dll
 0001:00000054       __imp__ExpandEnvironmentStringsW@12 10001054     kernel32:KERNEL32.dll
 0001:00000058       __imp__LocalFree@4         10001058     kernel32:KERNEL32.dll
 0001:0000005c       __imp__GetStringTypeW@16   1000105c     kernel32:KERNEL32.dll
 0001:00000060       __imp__LCMapStringW@24     10001060     kernel32:KERNEL32.dll
 0001:00000064       __imp__GetCurrentProcess@0 10001064     kernel32:KERNEL32.dll
 0001:00000068       __imp__TerminateProcess@8  10001068     kernel32:KERNEL32.dll
 0001:0000006c       __imp__IsDebuggerPresent@0 1000106c     kernel32:KERNEL32.dll
 0001:00000070       __imp__SetUnhandledExceptionFilter@4 10001070     kernel32:KERNEL32.dll
 0001:00000074       __imp__UnhandledExceptionFilter@4 10001074     kernel32:KERNEL32.dll
 0001:00000078       __imp__LoadLibraryW@4      10001078     kernel32:KERNEL32.dll
 0001:0000007c       __imp__HeapReAlloc@16      1000107c     kernel32:KERNEL32.dll
 0001:00000080       __imp__IsValidCodePage@4   10001080     kernel32:KERNEL32.dll
 0001:00000084       __imp__GetOEMCP@0          10001084     kernel32:KERNEL32.dll
 0001:00000088       __imp__GetACP@0            10001088     kernel32:KERNEL32.dll
 0001:0000008c       __imp__GetCPInfo@8         1000108c     kernel32:KERNEL32.dll
 0001:00000090       __imp__EnterCriticalSection@4 10001090     kernel32:KERNEL32.dll
 0001:00000094       __imp__LeaveCriticalSection@4 10001094     kernel32:KERNEL32.dll
 0001:00000098       __imp__GetModuleFileNameW@12 10001098     kernel32:KERNEL32.dll
 0001:0000009c       __imp__WriteFile@20        1000109c     kernel32:KERNEL32.dll
 0001:000000a0       __imp__HeapSize@12         100010a0     kernel32:KERNEL32.dll
 0001:000000a4       __imp__GetSystemTimeAsFileTime@4 100010a4     kernel32:KERNEL32.dll
 0001:000000a8       __imp__GetCurrentThreadId@0 100010a8     kernel32:KERNEL32.dll
 0001:000000ac       __imp__DecodePointer@4     100010ac     kernel32:KERNEL32.dll
 0001:000000b0       __imp__GetCommandLineA@0   100010b0     kernel32:KERNEL32.dll
 0001:000000b4       __imp__EncodePointer@4     100010b4     kernel32:KERNEL32.dll
 0001:000000b8       __imp__HeapAlloc@12        100010b8     kernel32:KERNEL32.dll
 0001:000000bc       __imp__RaiseException@16   100010bc     kernel32:KERNEL32.dll
 0001:000000c0       __imp__GetLastError@0      100010c0     kernel32:KERNEL32.dll
 0001:000000c4       __imp__HeapFree@12         100010c4     kernel32:KERNEL32.dll
 0001:000000c8       __imp__IsProcessorFeaturePresent@4 100010c8     kernel32:KERNEL32.dll
 0001:000000cc       __imp__RtlUnwind@16        100010cc     kernel32:KERNEL32.dll
 0001:000000d0       __imp__VirtualQuery@12     100010d0     kernel32:KERNEL32.dll
 0001:000000d4       __imp__TlsAlloc@0          100010d4     kernel32:KERNEL32.dll
 0001:000000d8       __imp__TlsGetValue@4       100010d8     kernel32:KERNEL32.dll
 0001:000000dc       __imp__TlsSetValue@8       100010dc     kernel32:KERNEL32.dll
 0001:000000e0       __imp__TlsFree@4           100010e0     kernel32:KERNEL32.dll
 0001:000000e4       __imp__InterlockedIncrement@4 100010e4     kernel32:KERNEL32.dll
 0001:000000e8       __imp__SetLastError@4      100010e8     kernel32:KERNEL32.dll
 0001:000000ec       __imp__InterlockedDecrement@4 100010ec     kernel32:KERNEL32.dll
 0001:000000f0       __imp__GetProcAddress@8    100010f0     kernel32:KERNEL32.dll
 0001:000000f4       __imp__Sleep@4             100010f4     kernel32:KERNEL32.dll
 0001:000000f8       __imp__ExitProcess@4       100010f8     kernel32:KERNEL32.dll
 0001:000000fc       __imp__SetHandleCount@4    100010fc     kernel32:KERNEL32.dll
 0001:00000100       __imp__GetStdHandle@4      10001100     kernel32:KERNEL32.dll
 0001:00000104       __imp__InitializeCriticalSectionAndSpinCount@8 10001104     kernel32:KERNEL32.dll
 0001:00000108       __imp__GetFileType@4       10001108     kernel32:KERNEL32.dll
 0001:0000010c       __imp__GetStartupInfoW@4   1000110c     kernel32:KERNEL32.dll
 0001:00000110       __imp__DeleteCriticalSection@4 10001110     kernel32:KERNEL32.dll
 0001:00000114       __imp__GetModuleFileNameA@12 10001114     kernel32:KERNEL32.dll
 0001:00000118       __imp__FreeEnvironmentStringsW@4 10001118     kernel32:KERNEL32.dll
 0001:0000011c       __imp__WideCharToMultiByte@32 1000111c     kernel32:KERNEL32.dll
 0001:00000120       __imp__GetEnvironmentStringsW@0 10001120     kernel32:KERNEL32.dll
 0001:00000124       __imp__HeapCreate@12       10001124     kernel32:KERNEL32.dll
 0001:00000128       __imp__HeapDestroy@4       10001128     kernel32:KERNEL32.dll
 0001:0000012c       __imp__QueryPerformanceCounter@4 1000112c     kernel32:KERNEL32.dll
 0001:00000130       __imp__GetTickCount@0      10001130     kernel32:KERNEL32.dll
 0001:00000134       __imp__GetCurrentProcessId@0 10001134     kernel32:KERNEL32.dll
 0001:00000138       \177KERNEL32_NULL_THUNK_DATA 10001138     kernel32:KERNEL32.dll
 0001:0000013c       __imp__SHGetSpecialFolderLocation@12 1000113c     shell32:SHELL32.dll
 0001:00000140       __imp__SHGetDesktopFolder@4 10001140     shell32:SHELL32.dll
 0001:00000144       \177SHELL32_NULL_THUNK_DATA 10001144     shell32:SHELL32.dll
 0001:00000148       __imp__GetMenuStringW@20   10001148     user32:USER32.dll
 0001:0000014c       __imp__GetWindowRect@8     1000114c     user32:USER32.dll
 0001:00000150       __imp__CreateDialogParamW@20 10001150     user32:USER32.dll
 0001:00000154       __imp__SetWindowPos@28     10001154     user32:USER32.dll
 0001:00000158       __imp__TrackPopupMenu@28   10001158     user32:USER32.dll
 0001:0000015c       __imp__GetMenuItemCount@4  1000115c     user32:USER32.dll
 0001:00000160       __imp__DestroyMenu@4       10001160     user32:USER32.dll
 0001:00000164       __imp__GetMenuItemInfoW@16 10001164     user32:USER32.dll
 0001:00000168       __imp__GetMessageW@16      10001168     user32:USER32.dll
 0001:0000016c       __imp__PeekMessageW@20     1000116c     user32:USER32.dll
 0001:00000170       __imp__DispatchMessageW@4  10001170     user32:USER32.dll
 0001:00000174       __imp__ReplyMessage@4      10001174     user32:USER32.dll
 0001:00000178       __imp__GetWindowLongW@8    10001178     user32:USER32.dll
 0001:0000017c       __imp__SetWindowLongW@12   1000117c     user32:USER32.dll
 0001:00000180       __imp__GetCursorPos@4      10001180     user32:USER32.dll
 0001:00000184       __imp__ScreenToClient@8    10001184     user32:USER32.dll
 0001:00000188       __imp__GetClientRect@8     10001188     user32:USER32.dll
 0001:0000018c       __imp__GetKeyState@4       1000118c     user32:USER32.dll
 0001:00000190       __imp__CreatePopupMenu@0   10001190     user32:USER32.dll
 0001:00000194       __imp__wsprintfW           10001194     user32:USER32.dll
 0001:00000198       __imp__DestroyWindow@4     10001198     user32:USER32.dll
 0001:0000019c       \177USER32_NULL_THUNK_DATA 1000119c     user32:USER32.dll
 0001:000001a0       __imp__CoTaskMemFree@4     100011a0     ole32:ole32.dll
 0001:000001a4       __imp__OleFlushClipboard@0 100011a4     ole32:ole32.dll
 0001:000001a8       __imp__OleInitialize@4     100011a8     ole32:ole32.dll
 0001:000001ac       \177ole32_NULL_THUNK_DATA  100011ac     ole32:ole32.dll
 0001:000001b0       ___xc_a                    100011b0     LIBCMT:crt0init.obj
 0001:000001b4       ___xc_z                    100011b4     LIBCMT:crt0init.obj
 0001:000001b8       ___xi_a                    100011b8     LIBCMT:crt0init.obj
 0001:000001c8       ___xi_z                    100011c8     LIBCMT:crt0init.obj
 0001:000001cc       ___xp_a                    100011cc     LIBCMT:crt0init.obj
 0001:000001d0       ___xp_z                    100011d0     LIBCMT:crt0init.obj
 0001:000001d4       ___xt_a                    100011d4     LIBCMT:crt0init.obj
 0001:000001d8       ___xt_z                    100011d8     LIBCMT:crt0init.obj
 0001:000001e0       _MainGuid                  100011e0     EMenu.obj
 0001:000001f0       _MenuGuid                  100011f0     EMenu.obj
 0001:00000200       _DialogGuid                10001200     EMenu.obj
 0001:00000210       _GuiTextMenuGuid           10001210     EMenu.obj
 0001:00000220       ??_C@_1DE@BGKMIKPD@?$AAE?$AAu?$AAg?$AAe?$AAn?$AAe?$AA?5?$AAR?$AAo?$AAs?$AAh?$AAa?$AAl?$AA?5?$AA?$CG?$AA?5?$AAF?$AAa?$AAr?$AA?5?$AAG?$AAr?$AAo?$AAu?$AAp?$AA?$AA@ 10001220     EMenu.obj
 0001:00000254       ??_C@_1DK@JMMNGKID@?$AAE?$AAM?$AAe?$AAn?$AAu?$AA?5?$AAP?$AAl?$AAu?$AAg?$AAi?$AAn?$AA?5?$AAf?$AAo?$AAr?$AA?5?$AAF?$AAa?$AAr?$AA?5?$AAM?$AAa?$AAn?$AAa?$AAg?$AAe?$AAr?$AA?$AA@ 10001254     EMenu.obj
 0001:00000290       ??_C@_1M@LBLKOFDL@?$AAE?$AAM?$AAe?$AAn?$AAu?$AA?$AA@ 10001290     EMenu.obj
 0001:000002a0       ??_C@_17CIEOGNAD@?$AA?5?$AA?5?$CF?$LK?$AA?$AA@ 100012a0     FarMenu.obj
 0001:000002a8       ??_C@_13HOIJIPNN@?$AA?5?$AA?$AA@ 100012a8     FarMenu.obj
 0001:000002ac       ??_C@_1M@IAIJHCCH@?$AAC?$AAl?$AAo?$AAs?$AAe?$AA?$AA@ 100012ac     Plugin.obj
 0001:000002b8       ??_C@_1O@MEJAHLJN@?$AAE?$AAr?$AAr?$AAo?$AAr?$AA2?$AA?$AA@ 100012b8     Plugin.obj
 0001:000002c8       ??_C@_1O@NGCFNEHD@?$AAE?$AAr?$AAr?$AAo?$AAr?$AA1?$AA?$AA@ 100012c8     Plugin.obj
 0001:000002d8       ??_C@_1O@GOJJLDBG@?$AAE?$AAr?$AAr?$AAo?$AAr?$AA0?$AA?$AA@ 100012d8     Plugin.obj
 0001:000002e8       ??_C@_1O@MCPHAIFL@?$AAM?$AAy?$AAC?$AAo?$AAm?$AAp?$AA?$AA@ 100012e8     Plugin.obj
 0001:000002f8       ??_C@_1BI@GILJGMBA@?$AAC?$AAo?$AAn?$AAt?$AAe?$AAx?$AAt?$AAM?$AAe?$AAn?$AAu?$AA?$AA@ 100012f8     Plugin.obj
 0001:00000310       ??_C@_1BO@CLHFIDDE@?$AAC?$AAh?$AAo?$AAo?$AAs?$AAe?$AAM?$AAe?$AAn?$AAu?$AAT?$AAy?$AAp?$AAe?$AA?$AA@ 10001310     Plugin.obj
 0001:00000330       ??_C@_1O@BJPKKLLM@?$AAC?$AAo?$AAn?$AAf?$AAi?$AAg?$AA?$AA@ 10001330     Plugin.obj
 0001:00000340       ??_C@_19JPHCGFBO@?$AAM?$AAa?$AAi?$AAn?$AA?$AA@ 10001340     Plugin.obj
 0001:0000034c       ??_C@_15DDHGOCBH@?$AA?4?$AA?4?$AA?$AA@ 1000134c     Plugin.obj
 0001:00000354       ??_7?$DialogBuilderBase@UFarDialogItem@@@@6B@ 10001354     Plugin.obj
 0001:00000378       __GUID_000214f4_0000_0000_c000_000000000046 10001378     Plugin.obj
 0001:00000388       __GUID_bcfce0a0_ec17_11d0_8d10_00a0c90f2719 10001388     Plugin.obj
 0001:00000398       ??_7PluginDialogBuilder@@6B@ 10001398     Plugin.obj
 0001:000003bc       ??_7?$DialogItemBinding@UFarDialogItem@@@@6B@ 100013bc     Plugin.obj
 0001:000003c4       ??_7PluginCheckBoxBinding@@6B@ 100013c4     Plugin.obj
 0001:000003cc       ??_7PluginRadioButtonBinding@@6B@ 100013cc     Plugin.obj
 0001:000003d4       ??_C@_15EFLNJKHH@?$AA?$CF?$AAu?$AA?$AA@ 100013d4     Plugin.obj
 0001:000003dc       ??_7PluginIntEditFieldBinding@@6B@ 100013dc     Plugin.obj
 0001:000003e4       ??_7PluginUIntEditFieldBinding@@6B@ 100013e4     Plugin.obj
 0001:000003ec       ??_C@_1O@EOCFEDGM@?$AAG?$AAu?$AAi?$AAP?$AAo?$AAs?$AA?$AA@ 100013ec     Plugin.obj
 0001:000003fc       ??_C@_1BM@JNPKPLGJ@?$AAD?$AAi?$AAf?$AAf?$AAe?$AAr?$AAe?$AAn?$AAt?$AAO?$AAn?$AAl?$AAy?$AA?$AA@ 100013fc     Plugin.obj
 0001:00000418       ??_C@_1BC@JAMHBCOF@?$AAH?$AAe?$AAl?$AAp?$AAt?$AAe?$AAx?$AAt?$AA?$AA@ 10001418     Plugin.obj
 0001:0000042c       ??_C@_1O@EFKGCNCH@?$AAS?$AAi?$AAl?$AAe?$AAn?$AAt?$AA?$AA@ 1000142c     Plugin.obj
 0001:0000043c       ??_C@_1BO@ELNGBDOB@?$AAC?$AAl?$AAe?$AAa?$AAr?$AAS?$AAe?$AAl?$AAe?$AAc?$AAt?$AAi?$AAo?$AAn?$AA?$AA@ 1000143c     Plugin.obj
 0001:0000045c       ??_C@_1BI@FNELDPIH@?$AAD?$AAe?$AAl?$AAU?$AAs?$AAi?$AAn?$AAg?$AAF?$AAa?$AAr?$AA?$AA@ 1000145c     Plugin.obj
 0001:00000474       ??_C@_1O@HAPBPKPP@?$AAU?$AAs?$AAe?$AAG?$AAU?$AAI?$AA?$AA@ 10001474     Plugin.obj
 0001:00000484       ??_C@_1BO@BLHAFJIH@?$AAW?$AAa?$AAi?$AAt?$AAT?$AAo?$AAC?$AAo?$AAn?$AAt?$AAi?$AAn?$AAu?$AAe?$AA?$AA@ 10001484     Plugin.obj
 0001:000004a8       ??_C@_1FE@DFGJMLLI@?$AAr?$AAc?$AAl?$AAk?$AA?3?$AAr?$AAc?$AAl?$AAk?$AA_?$AAt?$AAx?$AAt?$AA?3?$AAr?$AAc?$AAl?$AAk?$AA_?$AAg?$AAu?$AAi?$AA?3?$AAr?$AAc?$AAl?$AAk?$AA_?$AAc?$AAm?$AAd?$AA?3@ 100014a8     Plugin.obj
 0001:000004fc       ??_C@_11LOCGONAA@?$AA?$AA@ 100014fc     Plugin.obj
 0001:00000500       ??_C@_13DIBMAFH@?$AA?$CJ?$AA?$AA@ 10001500     Plugin.obj
 0001:00000504       ??_C@_15CMBHNMLL@?$AA?5?$AA?$CI?$AA?$AA@ 10001504     Plugin.obj
 0001:0000050c       ??_C@_1BO@PGPCBEEA@?$AAK?$AAe?$AAy?$AAs?$AA?8?$AAS?$AAh?$AAi?$AAf?$AAt?$AAD?$AAe?$AAl?$AA?8?$AA?$AA@ 1000150c     Plugin.obj
 0001:0000052c       ??_C@_1BK@NGCLJGHJ@?$AAK?$AAe?$AAy?$AAs?$AA?8?$AAA?$AAl?$AAt?$AAD?$AAe?$AAl?$AA?8?$AA?$AA@ 1000152c     Plugin.obj
 0001:00000548       ??_C@_1BC@BMPELNKI@?$AAK?$AAe?$AAy?$AAs?$AA?8?$AAF?$AA8?$AA?8?$AA?$AA@ 10001548     Plugin.obj
 0001:0000055c       ??_C@_06FOBLBEIN@delete?$AA@ 1000155c     Plugin.obj
 0001:00000564       ??_C@_1BC@CGPONMNI@?$AAK?$AAe?$AAy?$AAs?$AA?8?$AAF?$AA6?$AA?8?$AA?$AA@ 10001564     Plugin.obj
 0001:00000578       ??_C@_06LMEAOBLB@rename?$AA@ 10001578     Plugin.obj
 0001:00000580       ??_C@_15JOGBDECP@?$AA?0?$AA?5?$AA?$AA@ 10001580     Plugin.obj
 0001:00000588       ??_C@_1M@MDEFCCAF@?$AA?$CF?$AAu?$AA?5?$AA?$CF?$AAs?$AA?$AA@ 10001588     Plugin.obj
 0001:00000594       ??_C@_13FPGAJAPJ@?$AA?2?$AA?$AA@ 10001594     Plugin.obj
 0001:00000598       ??_C@_1BG@CJEHAOD@?$AAr?$AAc?$AAl?$AAk?$AA_?$AAi?$AAt?$AAe?$AAm?$AA?3?$AA?$AA@ 10001598     Plugin.obj
 0001:000005b0       ??_C@_1BE@JGMPCMJC@?$AAr?$AAc?$AAl?$AAk?$AA_?$AAc?$AAm?$AAd?$AA?3?$AA?$AA@ 100015b0     Plugin.obj
 0001:000005c4       ??_C@_1BE@IMOELFKI@?$AAr?$AAc?$AAl?$AAk?$AA_?$AAg?$AAu?$AAi?$AA?3?$AA?$AA@ 100015c4     Plugin.obj
 0001:000005d8       ??_C@_1BE@GEDAILNH@?$AAr?$AAc?$AAl?$AAk?$AA_?$AAt?$AAx?$AAt?$AA?3?$AA?$AA@ 100015d8     Plugin.obj
 0001:000005ec       ??_C@_1M@MGKMLCA@?$AAr?$AAc?$AAl?$AAk?$AA?3?$AA?$AA@ 100015ec     Plugin.obj
 0001:000005f8       _IID_IContextMenu          100015f8     shell32:shguid.obj
 0001:00000608       _IID_IShellFolder          10001608     shell32:shguid.obj
 0001:00000618       _IID_IDropTarget           10001618     uuid:oleidl_i.obj
 0001:00000628       _IID_IDataObject           10001628     uuid:objidl_i.obj
 0001:0000063c       ??_7bad_alloc@std@@6B@     1000163c     LIBCMT:new.obj
 0001:00000644       ??_C@_0P@GHFPNOJB@bad?5allocation?$AA@ 10001644     LIBCMT:new.obj
 0001:00000654       __pRawDllMain              10001654     LIBCMT:dllcrt0.obj
 0001:00000654       __pDefaultRawDllMain       10001654     LIBCMT:dllcrt0.obj
 0001:0000065c       ??_7exception@std@@6B@     1000165c     LIBCMT:stdexcpt.obj
 0001:00000664       ??_C@_0BC@EOODALEL@Unknown?5exception?$AA@ 10001664     LIBCMT:stdexcpt.obj
 0001:0000067c       ??_7type_info@@6B@         1000167c     LIBCMT:typinfo.obj
 0001:000006a0       ??_C@_1BK@DBDEIDLH@?$AAK?$AAE?$AAR?$AAN?$AAE?$AAL?$AA3?$AA2?$AA?4?$AAD?$AAL?$AAL?$AA?$AA@ 100016a0     LIBCMT:tidtable.obj
 0001:000006bc       ??_C@_07PEJMOBNF@FlsFree?$AA@ 100016bc     LIBCMT:tidtable.obj
 0001:000006c4       ??_C@_0M@JCPCPOEF@FlsSetValue?$AA@ 100016c4     LIBCMT:tidtable.obj
 0001:000006d0       ??_C@_0M@GDNOONDI@FlsGetValue?$AA@ 100016d0     LIBCMT:tidtable.obj
 0001:000006dc       ??_C@_08KNHFBNJ@FlsAlloc?$AA@ 100016dc     LIBCMT:tidtable.obj
 0001:000006e8       ??_C@_0P@MIGLKIOC@CorExitProcess?$AA@ 100016e8     LIBCMT:crt0dat.obj
 0001:000006f8       ??_C@_1BI@BGOHAHKC@?$AAm?$AAs?$AAc?$AAo?$AAr?$AAe?$AAe?$AA?4?$AAd?$AAl?$AAl?$AA?$AA@ 100016f8     LIBCMT:crt0dat.obj
 0001:00000710       __XcptActTab               10001710     LIBCMT:winxfltr.obj
 0001:000007a0       __First_FPE_Indx           100017a0     LIBCMT:winxfltr.obj
 0001:000007a4       __Num_FPE                  100017a4     LIBCMT:winxfltr.obj
 0001:000007a8       __XcptActTabSize           100017a8     LIBCMT:winxfltr.obj
 0001:000007ac       __XcptActTabCount          100017ac     LIBCMT:winxfltr.obj
 0001:000007b0       ??_C@_1BO@BKOMIGKJ@?$AAr?$AAu?$AAn?$AAt?$AAi?$AAm?$AAe?$AA?5?$AAe?$AAr?$AAr?$AAo?$AAr?$AA?5?$AA?$AA@ 100017b0     LIBCMT:crt0msg.obj
 0001:000007d0       ??_C@_15JNBOKNOG@?$AA?$AN?$AA?6?$AA?$AA@ 100017d0     LIBCMT:crt0msg.obj
 0001:000007d8       ??_C@_1BM@JBBEPPHI@?$AAT?$AAL?$AAO?$AAS?$AAS?$AA?5?$AAe?$AAr?$AAr?$AAo?$AAr?$AA?$AN?$AA?6?$AA?$AA@ 100017d8     LIBCMT:crt0msg.obj
 0001:000007f4       ??_C@_1BK@KMOMNAAI@?$AAS?$AAI?$AAN?$AAG?$AA?5?$AAe?$AAr?$AAr?$AAo?$AAr?$AA?$AN?$AA?6?$AA?$AA@ 100017f4     LIBCMT:crt0msg.obj
 0001:00000810       ??_C@_1BO@BFCDCGC@?$AAD?$AAO?$AAM?$AAA?$AAI?$AAN?$AA?5?$AAe?$AAr?$AAr?$AAo?$AAr?$AA?$AN?$AA?6?$AA?$AA@ 10001810     LIBCMT:crt0msg.obj
 0001:00000830       ??_C@_1BOO@KGEDBGAJ@?$AAR?$AA6?$AA0?$AA3?$AA3?$AA?$AN?$AA?6?$AA?9?$AA?5?$AAA?$AAt?$AAt?$AAe?$AAm?$AAp?$AAt?$AA?5?$AAt?$AAo?$AA?5?$AAu?$AAs?$AAe?$AA?5?$AAM?$AAS?$AAI?$AAL?$AA?5?$AAc?$AAo?$AAd@ 10001830     LIBCMT:crt0msg.obj
 0001:00000a20       ??_C@_1GG@GOPILAJP@?$AAR?$AA6?$AA0?$AA3?$AA2?$AA?$AN?$AA?6?$AA?9?$AA?5?$AAn?$AAo?$AAt?$AA?5?$AAe?$AAn?$AAo?$AAu?$AAg?$AAh?$AA?5?$AAs?$AAp?$AAa?$AAc?$AAe?$AA?5?$AAf?$AAo?$AAr?$AA?5?$AAl?$AAo@ 10001a20     LIBCMT:crt0msg.obj
 0001:00000a88       ??_C@_1MG@ENCOOIDF@?$AAR?$AA6?$AA0?$AA3?$AA1?$AA?$AN?$AA?6?$AA?9?$AA?5?$AAA?$AAt?$AAt?$AAe?$AAm?$AAp?$AAt?$AA?5?$AAt?$AAo?$AA?5?$AAi?$AAn?$AAi?$AAt?$AAi?$AAa?$AAl?$AAi?$AAz?$AAe?$AA?5?$AAt@ 10001a88     LIBCMT:crt0msg.obj
 0001:00000b50       ??_C@_1DO@BMFCDCD@?$AAR?$AA6?$AA0?$AA3?$AA0?$AA?$AN?$AA?6?$AA?9?$AA?5?$AAC?$AAR?$AAT?$AA?5?$AAn?$AAo?$AAt?$AA?5?$AAi?$AAn?$AAi?$AAt?$AAi?$AAa?$AAl?$AAi?$AAz?$AAe?$AAd?$AA?$AN?$AA?6?$AA?$AA@ 10001b50     LIBCMT:crt0msg.obj
 0001:00000b90       ??_C@_1EK@HHFLMAOL@?$AAR?$AA6?$AA0?$AA2?$AA8?$AA?$AN?$AA?6?$AA?9?$AA?5?$AAu?$AAn?$AAa?$AAb?$AAl?$AAe?$AA?5?$AAt?$AAo?$AA?5?$AAi?$AAn?$AAi?$AAt?$AAi?$AAa?$AAl?$AAi?$AAz?$AAe?$AA?5?$AAh?$AAe@ 10001b90     LIBCMT:crt0msg.obj
 0001:00000be0       ??_C@_1GK@MFGOKLAG@?$AAR?$AA6?$AA0?$AA2?$AA7?$AA?$AN?$AA?6?$AA?9?$AA?5?$AAn?$AAo?$AAt?$AA?5?$AAe?$AAn?$AAo?$AAu?$AAg?$AAh?$AA?5?$AAs?$AAp?$AAa?$AAc?$AAe?$AA?5?$AAf?$AAo?$AAr?$AA?5?$AAl?$AAo@ 10001be0     LIBCMT:crt0msg.obj
 0001:00000c50       ??_C@_1GK@MCAAGJMO@?$AAR?$AA6?$AA0?$AA2?$AA6?$AA?$AN?$AA?6?$AA?9?$AA?5?$AAn?$AAo?$AAt?$AA?5?$AAe?$AAn?$AAo?$AAu?$AAg?$AAh?$AA?5?$AAs?$AAp?$AAa?$AAc?$AAe?$AA?5?$AAf?$AAo?$AAr?$AA?5?$AAs?$AAt@ 10001c50     LIBCMT:crt0msg.obj
 0001:00000cc0       ??_C@_1EM@MAADIHMB@?$AAR?$AA6?$AA0?$AA2?$AA5?$AA?$AN?$AA?6?$AA?9?$AA?5?$AAp?$AAu?$AAr?$AAe?$AA?5?$AAv?$AAi?$AAr?$AAt?$AAu?$AAa?$AAl?$AA?5?$AAf?$AAu?$AAn?$AAc?$AAt?$AAi?$AAo?$AAn?$AA?5?$AAc@ 10001cc0     LIBCMT:crt0msg.obj
 0001:00000d10       ??_C@_1GK@FHCKBEFA@?$AAR?$AA6?$AA0?$AA2?$AA4?$AA?$AN?$AA?6?$AA?9?$AA?5?$AAn?$AAo?$AAt?$AA?5?$AAe?$AAn?$AAo?$AAu?$AAg?$AAh?$AA?5?$AAs?$AAp?$AAa?$AAc?$AAe?$AA?5?$AAf?$AAo?$AAr?$AA?5?$AA_?$AAo@ 10001d10     LIBCMT:crt0msg.obj
 0001:00000d80       ??_C@_1FC@ECHBIFBC@?$AAR?$AA6?$AA0?$AA1?$AA9?$AA?$AN?$AA?6?$AA?9?$AA?5?$AAu?$AAn?$AAa?$AAb?$AAl?$AAe?$AA?5?$AAt?$AAo?$AA?5?$AAo?$AAp?$AAe?$AAn?$AA?5?$AAc?$AAo?$AAn?$AAs?$AAo?$AAl?$AAe?$AA?5@ 10001d80     LIBCMT:crt0msg.obj
 0001:00000dd8       ??_C@_1EC@JIBHAOPH@?$AAR?$AA6?$AA0?$AA1?$AA8?$AA?$AN?$AA?6?$AA?9?$AA?5?$AAu?$AAn?$AAe?$AAx?$AAp?$AAe?$AAc?$AAt?$AAe?$AAd?$AA?5?$AAh?$AAe?$AAa?$AAp?$AA?5?$AAe?$AAr?$AAr?$AAo?$AAr?$AA?$AN?$AA?6@ 10001dd8     LIBCMT:crt0msg.obj
 0001:00000e20       ??_C@_1FK@BEOGODMC@?$AAR?$AA6?$AA0?$AA1?$AA7?$AA?$AN?$AA?6?$AA?9?$AA?5?$AAu?$AAn?$AAe?$AAx?$AAp?$AAe?$AAc?$AAt?$AAe?$AAd?$AA?5?$AAm?$AAu?$AAl?$AAt?$AAi?$AAt?$AAh?$AAr?$AAe?$AAa?$AAd?$AA?5@ 10001e20     LIBCMT:crt0msg.obj
 0001:00000e80       ??_C@_1FI@LOGNIKDM@?$AAR?$AA6?$AA0?$AA1?$AA6?$AA?$AN?$AA?6?$AA?9?$AA?5?$AAn?$AAo?$AAt?$AA?5?$AAe?$AAn?$AAo?$AAu?$AAg?$AAh?$AA?5?$AAs?$AAp?$AAa?$AAc?$AAe?$AA?5?$AAf?$AAo?$AAr?$AA?5?$AAt?$AAh@ 10001e80     LIBCMT:crt0msg.obj
 0001:00000ed8       ??_C@_1EG@BEHAGFJD@?$AAR?$AA6?$AA0?$AA1?$AA0?$AA?$AN?$AA?6?$AA?9?$AA?5?$AAa?$AAb?$AAo?$AAr?$AAt?$AA?$CI?$AA?$CJ?$AA?5?$AAh?$AAa?$AAs?$AA?5?$AAb?$AAe?$AAe?$AAn?$AA?5?$AAc?$AAa?$AAl?$AAl?$AAe?$AAd@ 10001ed8     LIBCMT:crt0msg.obj
 0001:00000f20       ??_C@_1FI@HONFMGBI@?$AAR?$AA6?$AA0?$AA0?$AA9?$AA?$AN?$AA?6?$AA?9?$AA?5?$AAn?$AAo?$AAt?$AA?5?$AAe?$AAn?$AAo?$AAu?$AAg?$AAh?$AA?5?$AAs?$AAp?$AAa?$AAc?$AAe?$AA?5?$AAf?$AAo?$AAr?$AA?5?$AAe?$AAn@ 10001f20     LIBCMT:crt0msg.obj
 0001:00000f78       ??_C@_1FE@LLNEDJMD@?$AAR?$AA6?$AA0?$AA0?$AA8?$AA?$AN?$AA?6?$AA?9?$AA?5?$AAn?$AAo?$AAt?$AA?5?$AAe?$AAn?$AAo?$AAu?$AAg?$AAh?$AA?5?$AAs?$AAp?$AAa?$AAc?$AAe?$AA?5?$AAf?$AAo?$AAr?$AA?5?$AAa?$AAr@ 10001f78     LIBCMT:crt0msg.obj
 0001:00000fd0       ??_C@_1FK@PGACCAFB@?$AAR?$AA6?$AA0?$AA0?$AA2?$AA?$AN?$AA?6?$AA?9?$AA?5?$AAf?$AAl?$AAo?$AAa?$AAt?$AAi?$AAn?$AAg?$AA?5?$AAp?$AAo?$AAi?$AAn?$AAt?$AA?5?$AAs?$AAu?$AAp?$AAp?$AAo?$AAr?$AAt?$AA?5@ 10001fd0     LIBCMT:crt0msg.obj
 0001:000010e0       ??_C@_1EK@MBDPDCGA@?$AAM?$AAi?$AAc?$AAr?$AAo?$AAs?$AAo?$AAf?$AAt?$AA?5?$AAV?$AAi?$AAs?$AAu?$AAa?$AAl?$AA?5?$AAC?$AA?$CL?$AA?$CL?$AA?5?$AAR?$AAu?$AAn?$AAt?$AAi?$AAm?$AAe?$AA?5?$AAL?$AAi?$AAb@ 100020e0     LIBCMT:crt0msg.obj
 0001:0000112c       ??_C@_15IABLJNFO@?$AA?6?$AA?6?$AA?$AA@ 1000212c     LIBCMT:crt0msg.obj
 0001:00001134       ??_C@_17LGKOMLJ@?$AA?4?$AA?4?$AA?4?$AA?$AA@ 10002134     LIBCMT:crt0msg.obj
 0001:0000113c       ??_C@_1CO@EAEJAADC@?$AA?$DM?$AAp?$AAr?$AAo?$AAg?$AAr?$AAa?$AAm?$AA?5?$AAn?$AAa?$AAm?$AAe?$AA?5?$AAu?$AAn?$AAk?$AAn?$AAo?$AAw?$AAn?$AA?$DO?$AA?$AA@ 1000213c     LIBCMT:crt0msg.obj
 0001:0000116c       ??_C@_1DE@JNGNBFGO@?$AAR?$AAu?$AAn?$AAt?$AAi?$AAm?$AAe?$AA?5?$AAE?$AAr?$AAr?$AAo?$AAr?$AA?$CB?$AA?6?$AA?6?$AAP?$AAr?$AAo?$AAg?$AAr?$AAa?$AAm?$AA?3?$AA?5?$AA?$AA@ 1000216c     LIBCMT:crt0msg.obj
 0001:000011a0       ??_C@_1BC@GDGBMEMK@?$AAH?$AAH?$AA?3?$AAm?$AAm?$AA?3?$AAs?$AAs?$AA?$AA@ 100021a0     LIBCMT:nlsdata2.obj
 0001:000011b4       ??_C@_1CI@KNAKOEBC@?$AAd?$AAd?$AAd?$AAd?$AA?0?$AA?5?$AAM?$AAM?$AAM?$AAM?$AA?5?$AAd?$AAd?$AA?0?$AA?5?$AAy?$AAy?$AAy?$AAy?$AA?$AA@ 100021b4     LIBCMT:nlsdata2.obj
 0001:000011dc       ??_C@_1BC@IEBCMHCM@?$AAM?$AAM?$AA?1?$AAd?$AAd?$AA?1?$AAy?$AAy?$AA?$AA@ 100021dc     LIBCMT:nlsdata2.obj
 0001:000011f0       ??_C@_15CLMNNGEL@?$AAP?$AAM?$AA?$AA@ 100021f0     LIBCMT:nlsdata2.obj
 0001:000011f8       ??_C@_15ODEHAHHF@?$AAA?$AAM?$AA?$AA@ 100021f8     LIBCMT:nlsdata2.obj
 0001:00001200       ??_C@_1BC@FEMKIFH@?$AAD?$AAe?$AAc?$AAe?$AAm?$AAb?$AAe?$AAr?$AA?$AA@ 10002200     LIBCMT:nlsdata2.obj
 0001:00001214       ??_C@_1BC@BGLIFPF@?$AAN?$AAo?$AAv?$AAe?$AAm?$AAb?$AAe?$AAr?$AA?$AA@ 10002214     LIBCMT:nlsdata2.obj
 0001:00001228       ??_C@_1BA@EPANDLNG@?$AAO?$AAc?$AAt?$AAo?$AAb?$AAe?$AAr?$AA?$AA@ 10002228     LIBCMT:nlsdata2.obj
 0001:00001238       ??_C@_1BE@DKAAMBJL@?$AAS?$AAe?$AAp?$AAt?$AAe?$AAm?$AAb?$AAe?$AAr?$AA?$AA@ 10002238     LIBCMT:nlsdata2.obj
 0001:0000124c       ??_C@_1O@PAHLKOAC@?$AAA?$AAu?$AAg?$AAu?$AAs?$AAt?$AA?$AA@ 1000224c     LIBCMT:nlsdata2.obj
 0001:0000125c       ??_C@_19BIFMLPCD@?$AAJ?$AAu?$AAl?$AAy?$AA?$AA@ 1000225c     LIBCMT:nlsdata2.obj
 0001:00001268       ??_C@_19EPFLPGAP@?$AAJ?$AAu?$AAn?$AAe?$AA?$AA@ 10002268     LIBCMT:nlsdata2.obj
 0001:00001274       ??_C@_1M@GJNLMHFD@?$AAA?$AAp?$AAr?$AAi?$AAl?$AA?$AA@ 10002274     LIBCMT:nlsdata2.obj
 0001:00001280       ??_C@_1M@IKEENEDF@?$AAM?$AAa?$AAr?$AAc?$AAh?$AA?$AA@ 10002280     LIBCMT:nlsdata2.obj
 0001:0000128c       ??_C@_1BC@JGDDFFAM@?$AAF?$AAe?$AAb?$AAr?$AAu?$AAa?$AAr?$AAy?$AA?$AA@ 1000228c     LIBCMT:nlsdata2.obj
 0001:000012a0       ??_C@_1BA@EFMEIEBA@?$AAJ?$AAa?$AAn?$AAu?$AAa?$AAr?$AAy?$AA?$AA@ 100022a0     LIBCMT:nlsdata2.obj
 0001:000012b0       ??_C@_17EGKACKIF@?$AAD?$AAe?$AAc?$AA?$AA@ 100022b0     LIBCMT:nlsdata2.obj
 0001:000012b8       ??_C@_17BBDMLCIG@?$AAN?$AAo?$AAv?$AA?$AA@ 100022b8     LIBCMT:nlsdata2.obj
 0001:000012c0       ??_C@_17FNLKOI@?$AAO?$AAc?$AAt?$AA?$AA@ 100022c0     LIBCMT:nlsdata2.obj
 0001:000012c8       ??_C@_17HCHCOKMG@?$AAS?$AAe?$AAp?$AA?$AA@ 100022c8     LIBCMT:nlsdata2.obj
 0001:000012d0       ??_C@_17ICPELBCN@?$AAA?$AAu?$AAg?$AA?$AA@ 100022d0     LIBCMT:nlsdata2.obj
 0001:000012d8       ??_C@_17IJPCKHK@?$AAJ?$AAu?$AAl?$AA?$AA@ 100022d8     LIBCMT:nlsdata2.obj
 0001:000012e0       ??_C@_17KCJGOCPB@?$AAJ?$AAu?$AAn?$AA?$AA@ 100022e0     LIBCMT:nlsdata2.obj
 0001:000012e8       ??_C@_17PNNKMEED@?$AAM?$AAa?$AAy?$AA?$AA@ 100022e8     LIBCMT:nlsdata2.obj
 0001:000012f0       ??_C@_17LFPOIHDD@?$AAA?$AAp?$AAr?$AA?$AA@ 100022f0     LIBCMT:nlsdata2.obj
 0001:000012f8       ??_C@_17CKNLEDEC@?$AAM?$AAa?$AAr?$AA?$AA@ 100022f8     LIBCMT:nlsdata2.obj
 0001:00001300       ??_C@_17LMDJEKJN@?$AAF?$AAe?$AAb?$AA?$AA@ 10002300     LIBCMT:nlsdata2.obj
 0001:00001308       ??_C@_17DKNBKCHM@?$AAJ?$AAa?$AAn?$AA?$AA@ 10002308     LIBCMT:nlsdata2.obj
 0001:00001310       ??_C@_1BC@ENMNNPAJ@?$AAS?$AAa?$AAt?$AAu?$AAr?$AAd?$AAa?$AAy?$AA?$AA@ 10002310     LIBCMT:nlsdata2.obj
 0001:00001324       ??_C@_1O@PDICJHAG@?$AAF?$AAr?$AAi?$AAd?$AAa?$AAy?$AA?$AA@ 10002324     LIBCMT:nlsdata2.obj
 0001:00001334       ??_C@_1BC@HHMNLIHE@?$AAT?$AAh?$AAu?$AAr?$AAs?$AAd?$AAa?$AAy?$AA?$AA@ 10002334     LIBCMT:nlsdata2.obj
 0001:00001348       ??_C@_1BE@EBOGMDOH@?$AAW?$AAe?$AAd?$AAn?$AAe?$AAs?$AAd?$AAa?$AAy?$AA?$AA@ 10002348     LIBCMT:nlsdata2.obj
 0001:0000135c       ??_C@_1BA@ENFBFFEK@?$AAT?$AAu?$AAe?$AAs?$AAd?$AAa?$AAy?$AA?$AA@ 1000235c     LIBCMT:nlsdata2.obj
 0001:0000136c       ??_C@_1O@MMNBFLIA@?$AAM?$AAo?$AAn?$AAd?$AAa?$AAy?$AA?$AA@ 1000236c     LIBCMT:nlsdata2.obj
 0001:0000137c       ??_C@_1O@IHNHDHPB@?$AAS?$AAu?$AAn?$AAd?$AAa?$AAy?$AA?$AA@ 1000237c     LIBCMT:nlsdata2.obj
 0001:0000138c       ??_C@_17GGIBDPIH@?$AAS?$AAa?$AAt?$AA?$AA@ 1000238c     LIBCMT:nlsdata2.obj
 0001:00001394       ??_C@_17HFOLPPLP@?$AAF?$AAr?$AAi?$AA?$AA@ 10002394     LIBCMT:nlsdata2.obj
 0001:0000139c       ??_C@_17PDPHAADD@?$AAT?$AAh?$AAu?$AA?$AA@ 1000239c     LIBCMT:nlsdata2.obj
 0001:000013a4       ??_C@_17CJEDCEPE@?$AAW?$AAe?$AAd?$AA?$AA@ 100023a4     LIBCMT:nlsdata2.obj
 0001:000013ac       ??_C@_17BMKGEGOJ@?$AAT?$AAu?$AAe?$AA?$AA@ 100023ac     LIBCMT:nlsdata2.obj
 0001:000013b4       ??_C@_17KBOMKBF@?$AAM?$AAo?$AAn?$AA?$AA@ 100023b4     LIBCMT:nlsdata2.obj
 0001:000013bc       ??_C@_17MBGCMIPB@?$AAS?$AAu?$AAn?$AA?$AA@ 100023bc     LIBCMT:nlsdata2.obj
 0001:000013c4       ??_C@_08JCCMCCIL@HH?3mm?3ss?$AA@ 100023c4     LIBCMT:nlsdata2.obj
 0001:000013d0       ??_C@_0BE@CKGJFCPC@dddd?0?5MMMM?5dd?0?5yyyy?$AA@ 100023d0     LIBCMT:nlsdata2.obj
 0001:000013e4       ??_C@_08BPBNCDIB@MM?1dd?1yy?$AA@ 100023e4     LIBCMT:nlsdata2.obj
 0001:000013f0       ??_C@_02CJNFDJBF@PM?$AA@   100023f0     LIBCMT:nlsdata2.obj
 0001:000013f4       ??_C@_02DEDBPAFC@AM?$AA@   100023f4     LIBCMT:nlsdata2.obj
 0001:000013f8       ??_C@_08EDHMEBNP@December?$AA@ 100023f8     LIBCMT:nlsdata2.obj
 0001:00001404       ??_C@_08HCHEGEOA@November?$AA@ 10002404     LIBCMT:nlsdata2.obj
 0001:00001410       ??_C@_07JJNFCEND@October?$AA@ 10002410     LIBCMT:nlsdata2.obj
 0001:00001418       ??_C@_09BHHEALKD@September?$AA@ 10002418     LIBCMT:nlsdata2.obj
 0001:00001424       ??_C@_06LBBHFDDG@August?$AA@ 10002424     LIBCMT:nlsdata2.obj
 0001:0000142c       ??_C@_04MIEPOIFP@July?$AA@ 1000242c     LIBCMT:nlsdata2.obj
 0001:00001434       ??_C@_04CNLMGBGM@June?$AA@ 10002434     LIBCMT:nlsdata2.obj
 0001:0000143c       ??_C@_05DMJDNLEJ@April?$AA@ 1000243c     LIBCMT:nlsdata2.obj
 0001:00001444       ??_C@_05HPCKOFNC@March?$AA@ 10002444     LIBCMT:nlsdata2.obj
 0001:0000144c       ??_C@_08GNJGEPFN@February?$AA@ 1000244c     LIBCMT:nlsdata2.obj
 0001:00001458       ??_C@_07CGJPFGJA@January?$AA@ 10002458     LIBCMT:nlsdata2.obj
 0001:00001460       ??_C@_03MKABNOCG@Dec?$AA@  10002460     LIBCMT:nlsdata2.obj
 0001:00001464       ??_C@_03JPJOFNIA@Nov?$AA@  10002464     LIBCMT:nlsdata2.obj
 0001:00001468       ??_C@_03BMAOKBAD@Oct?$AA@  10002468     LIBCMT:nlsdata2.obj
 0001:0000146c       ??_C@_03GGCAPAJC@Sep?$AA@  1000246c     LIBCMT:nlsdata2.obj
 0001:00001470       ??_C@_03IFJFEIGA@Aug?$AA@  10002470     LIBCMT:nlsdata2.obj
 0001:00001474       ??_C@_03LBGABGKK@Jul?$AA@  10002474     LIBCMT:nlsdata2.obj
 0001:00001478       ??_C@_03IDFGHECI@Jun?$AA@  10002478     LIBCMT:nlsdata2.obj
 0001:0000147c       ??_C@_03CNMDKL@May?$AA@    1000247c     LIBCMT:nlsdata2.obj
 0001:00001480       ??_C@_03LEOLGMJP@Apr?$AA@  10002480     LIBCMT:nlsdata2.obj
 0001:00001484       ??_C@_03ODNJBKGA@Mar?$AA@  10002484     LIBCMT:nlsdata2.obj
 0001:00001488       ??_C@_03HJBDCHOM@Feb?$AA@  10002488     LIBCMT:nlsdata2.obj
 0001:0000148c       ??_C@_03JIHJHPIE@Jan?$AA@  1000248c     LIBCMT:nlsdata2.obj
 0001:00001490       ??_C@_08INBOOONO@Saturday?$AA@ 10002490     LIBCMT:nlsdata2.obj
 0001:0000149c       ??_C@_06JECMNKMI@Friday?$AA@ 1000249c     LIBCMT:nlsdata2.obj
 0001:000014a4       ??_C@_08HACCIKIA@Thursday?$AA@ 100024a4     LIBCMT:nlsdata2.obj
 0001:000014b0       ??_C@_09DLIGFAKA@Wednesday?$AA@ 100024b0     LIBCMT:nlsdata2.obj
 0001:000014bc       ??_C@_07BAAGCFCM@Tuesday?$AA@ 100024bc     LIBCMT:nlsdata2.obj
 0001:000014c4       ??_C@_06JLEDEDGH@Monday?$AA@ 100024c4     LIBCMT:nlsdata2.obj
 0001:000014cc       ??_C@_06OOPIFAJ@Sunday?$AA@ 100024cc     LIBCMT:nlsdata2.obj
 0001:000014d4       ??_C@_03FEFJNEK@Sat?$AA@   100024d4     LIBCMT:nlsdata2.obj
 0001:000014d8       ??_C@_03IDIOELNC@Fri?$AA@  100024d8     LIBCMT:nlsdata2.obj
 0001:000014dc       ??_C@_03IOFIKPDN@Thu?$AA@  100024dc     LIBCMT:nlsdata2.obj
 0001:000014e0       ??_C@_03MHOMLAJA@Wed?$AA@  100024e0     LIBCMT:nlsdata2.obj
 0001:000014e4       ??_C@_03NAGEINEP@Tue?$AA@  100024e4     LIBCMT:nlsdata2.obj
 0001:000014e8       ??_C@_03PDAGKDH@Mon?$AA@   100024e8     LIBCMT:nlsdata2.obj
 0001:000014ec       ??_C@_03KOEHGMDN@Sun?$AA@  100024ec     LIBCMT:nlsdata2.obj
 0001:000014f0       ??_C@_0BK@CFCOFLF@?5Complete?5Object?5Locator?8?$AA@ 100024f0     LIBCMT:undname.obj
 0001:0000150c       ??_C@_0BN@MECKDCOJ@?5Class?5Hierarchy?5Descriptor?8?$AA@ 1000250c     LIBCMT:undname.obj
 0001:0000152c       ??_C@_0BD@LGICGFMM@?5Base?5Class?5Array?8?$AA@ 1000252c     LIBCMT:undname.obj
 0001:00001540       ??_C@_0BM@LDKODKLH@?5Base?5Class?5Descriptor?5at?5?$CI?$AA@ 10002540     LIBCMT:undname.obj
 0001:0000155c       ??_C@_0BC@DAFEJGAK@?5Type?5Descriptor?8?$AA@ 1000255c     LIBCMT:undname.obj
 0001:00001570       ??_C@_0BM@PMGGMLDN@?$GAlocal?5static?5thread?5guard?8?$AA@ 10002570     LIBCMT:undname.obj
 0001:0000158c       ??_C@_0CL@FGIJHLCE@?$GAmanaged?5vector?5copy?5constructor@ 1000258c     LIBCMT:undname.obj
 0001:000015b8       ??_C@_0CJ@GJELGAMM@?$GAvector?5vbase?5copy?5constructor?5i@ 100025b8     LIBCMT:undname.obj
 0001:000015e4       ??_C@_0CD@CGAJBKEJ@?$GAvector?5copy?5constructor?5iterato@ 100025e4     LIBCMT:undname.obj
 0001:00001608       ??_C@_0CB@PDBIFEP@?$GAdynamic?5atexit?5destructor?5for?5?8@ 10002608     LIBCMT:undname.obj
 0001:0000162c       ??_C@_0BL@CLIPGLGB@?$GAdynamic?5initializer?5for?5?8?$AA@ 1000262c     LIBCMT:undname.obj
 0001:00001648       ??_C@_0CM@FCBBDIGB@?$GAeh?5vector?5vbase?5copy?5constructo@ 10002648     LIBCMT:undname.obj
 0001:00001674       ??_C@_0CG@HLDDJMAG@?$GAeh?5vector?5copy?5constructor?5iter@ 10002674     LIBCMT:undname.obj
 0001:0000169c       ??_C@_0CF@IMGKMJNO@?$GAmanaged?5vector?5destructor?5itera@ 1000269c     LIBCMT:undname.obj
 0001:000016c4       ??_C@_0CG@CFDHKGGD@?$GAmanaged?5vector?5constructor?5iter@ 100026c4     LIBCMT:undname.obj
 0001:000016ec       ??_C@_0BN@CKNJLHMB@?$GAplacement?5delete?$FL?$FN?5closure?8?$AA@ 100026ec     LIBCMT:undname.obj
 0001:0000170c       ??_C@_0BL@CNOONJFP@?$GAplacement?5delete?5closure?8?$AA@ 1000270c     LIBCMT:undname.obj
 0001:00001728       ??_C@_0P@HJKNJFNN@?$GAomni?5callsig?8?$AA@ 10002728     LIBCMT:undname.obj
 0001:00001738       ??_C@_09LBNFPBCA@?5delete?$FL?$FN?$AA@ 10002738     LIBCMT:undname.obj
 0001:00001744       ??_C@_06FHBGPFGH@?5new?$FL?$FN?$AA@ 10002744     LIBCMT:undname.obj
 0001:0000174c       ??_C@_0CE@IIHCMGGL@?$GAlocal?5vftable?5constructor?5closu@ 1000274c     LIBCMT:undname.obj
 0001:00001770       ??_C@_0BA@KKLDJDLB@?$GAlocal?5vftable?8?$AA@ 10002770     LIBCMT:undname.obj
 0001:00001780       ??_C@_05KHLCHHI@?$GARTTI?$AA@ 10002780     LIBCMT:undname.obj
 0001:00001788       ??_C@_03KLGMFNMG@?$GAEH?$AA@ 10002788     LIBCMT:undname.obj
 0001:0000178c       ??_C@_0BA@KBCDOMBN@?$GAudt?5returning?8?$AA@ 1000278c     LIBCMT:undname.obj
 0001:0000179c       ??_C@_0BL@LLKPOHJI@?$GAcopy?5constructor?5closure?8?$AA@ 1000279c     LIBCMT:undname.obj
 0001:000017b8       ??_C@_0CH@OOJPLCPH@?$GAeh?5vector?5vbase?5constructor?5ite@ 100027b8     LIBCMT:undname.obj
 0001:000017e0       ??_C@_0CA@GCEOPDGL@?$GAeh?5vector?5destructor?5iterator?8?$AA@ 100027e0     LIBCMT:undname.obj
 0001:00001800       ??_C@_0CB@JONCMFFK@?$GAeh?5vector?5constructor?5iterator?8@ 10002800     LIBCMT:undname.obj
 0001:00001824       ??_C@_0BL@NILFHHPC@?$GAvirtual?5displacement?5map?8?$AA@ 10002824     LIBCMT:undname.obj
 0001:00001840       ??_C@_0CE@IKBNEHA@?$GAvector?5vbase?5constructor?5iterat@ 10002840     LIBCMT:undname.obj
 0001:00001864       ??_C@_0BN@LFPFMEDL@?$GAvector?5destructor?5iterator?8?$AA@ 10002864     LIBCMT:undname.obj
 0001:00001884       ??_C@_0BO@PFGOCPJJ@?$GAvector?5constructor?5iterator?8?$AA@ 10002884     LIBCMT:undname.obj
 0001:000018a4       ??_C@_0BN@IMDCHIKM@?$GAscalar?5deleting?5destructor?8?$AA@ 100028a4     LIBCMT:undname.obj
 0001:000018c4       ??_C@_0BO@OBMKPJIG@?$GAdefault?5constructor?5closure?8?$AA@ 100028c4     LIBCMT:undname.obj
 0001:000018e4       ??_C@_0BN@DEGPLNFK@?$GAvector?5deleting?5destructor?8?$AA@ 100028e4     LIBCMT:undname.obj
 0001:00001904       ??_C@_0BD@JDLKDPAB@?$GAvbase?5destructor?8?$AA@ 10002904     LIBCMT:undname.obj
 0001:00001918       ??_C@_08OBABFOLI@?$GAstring?8?$AA@ 10002918     LIBCMT:undname.obj
 0001:00001924       ??_C@_0BF@KDPPACIK@?$GAlocal?5static?5guard?8?$AA@ 10002924     LIBCMT:undname.obj
 0001:0000193c       ??_C@_08LLFFHHDJ@?$GAtypeof?8?$AA@ 1000293c     LIBCMT:undname.obj
 0001:00001948       ??_C@_07FEEIOKP@?$GAvcall?8?$AA@ 10002948     LIBCMT:undname.obj
 0001:00001950       ??_C@_09BLBHBJP@?$GAvbtable?8?$AA@ 10002950     LIBCMT:undname.obj
 0001:0000195c       ??_C@_09IFPLHPGF@?$GAvftable?8?$AA@ 1000295c     LIBCMT:undname.obj
 0001:00001968       ??_C@_02MHEGNOJ@?$FO?$DN?$AA@ 10002968     LIBCMT:undname.obj
 0001:0000196c       ??_C@_02DHLNPPGH@?$HM?$DN?$AA@ 1000296c     LIBCMT:undname.obj
 0001:00001970       ??_C@_02FGJGFEAB@?$CG?$DN?$AA@ 10002970     LIBCMT:undname.obj
 0001:00001974       ??_C@_03CDNPDDLA@?$DM?$DM?$DN?$AA@ 10002974     LIBCMT:undname.obj
 0001:00001978       ??_C@_03IKFCCPFF@?$DO?$DO?$DN?$AA@ 10002978     LIBCMT:undname.obj
 0001:0000197c       ??_C@_02FENAOKFI@?$CF?$DN?$AA@ 1000297c     LIBCMT:undname.obj
 0001:00001980       ??_C@_02FJEHGPIO@?1?$DN?$AA@ 10002980     LIBCMT:undname.obj
 0001:00001984       ??_C@_02FKMDLLOA@?9?$DN?$AA@ 10002984     LIBCMT:undname.obj
 0001:00001988       ??_C@_02FOEOMHFC@?$CL?$DN?$AA@ 10002988     LIBCMT:undname.obj
 0001:0000198c       ??_C@_02FPIMKNGF@?$CK?$DN?$AA@ 1000298c     LIBCMT:undname.obj
 0001:00001990       ??_C@_02NONPIBCD@?$HM?$HM?$AA@ 10002990     LIBCMT:undname.obj
 0001:00001994       ??_C@_02PPKAJPJL@?$CG?$CG?$AA@ 10002994     LIBCMT:undname.obj
 0001:00001998       ??_C@_01DNKMNLPK@?$HM?$AA@ 10002998     LIBCMT:undname.obj
 0001:0000199c       ??_C@_01JKBOJNNK@?$FO?$AA@ 1000299c     LIBCMT:undname.obj
 0001:000019a0       ??_C@_01PJKLJHI@?$HO?$AA@  100029a0     LIBCMT:undname.obj
 0001:000019a4       ??_C@_02HCKGKOFO@?$CI?$CJ?$AA@ 100029a4     LIBCMT:undname.obj
 0001:000019a8       ??_C@_01IHBHIGKO@?0?$AA@   100029a8     LIBCMT:undname.obj
 0001:000019ac       ??_C@_02EEKDKGMJ@?$DO?$DN?$AA@ 100029ac     LIBCMT:undname.obj
 0001:000019b0       ??_C@_01PPODPGHN@?$DO?$AA@ 100029b0     LIBCMT:undname.obj
 0001:000019b4       ??_C@_02EHCHHCKH@?$DM?$DN?$AA@ 100029b4     LIBCMT:undname.obj
 0001:000019b8       ??_C@_01MNNFJEPP@?$DM?$AA@ 100029b8     LIBCMT:undname.obj
 0001:000019bc       ??_C@_01FGNFDNOH@?$CF?$AA@ 100029bc     LIBCMT:undname.obj
 0001:000019c0       ??_C@_01KMDKNFGN@?1?$AA@   100029c0     LIBCMT:undname.obj
 0001:000019c4       ??_C@_03MNHNFDLC@?9?$DO?$CK?$AA@ 100029c4     LIBCMT:undname.obj
 0001:000019c8       ??_C@_01HNPIGOCE@?$CG?$AA@ 100029c8     LIBCMT:undname.obj
 0001:000019cc       ??_C@_01MIFGBAGJ@?$CL?$AA@ 100029cc     LIBCMT:undname.obj
 0001:000019d0       ??_C@_01JOAMLHOP@?9?$AA@   100029d0     LIBCMT:undname.obj
 0001:000019d4       ??_C@_02BAABKJLB@?9?9?$AA@ 100029d4     LIBCMT:undname.obj
 0001:000019d8       ??_C@_02ECNGHCIF@?$CL?$CL?$AA@ 100029d8     LIBCMT:undname.obj
 0001:000019dc       ??_C@_01NBENCBCI@?$CK?$AA@ 100029dc     LIBCMT:undname.obj
 0001:000019e0       ??_C@_02HBOOOICD@?9?$DO?$AA@ 100029e0     LIBCMT:undname.obj
 0001:000019e4       ??_C@_08LHJFAFGD@operator?$AA@ 100029e4     LIBCMT:undname.obj
 0001:000019f0       ??_C@_02GPECMEKF@?$FL?$FN?$AA@ 100029f0     LIBCMT:undname.obj
 0001:000019f4       ??_C@_02FDNJECIE@?$CB?$DN?$AA@ 100029f4     LIBCMT:undname.obj
 0001:000019f8       ??_C@_02EGOFBIJA@?$DN?$DN?$AA@ 100029f8     LIBCMT:undname.obj
 0001:000019fc       ??_C@_01DCLJPIOD@?$CB?$AA@ 100029fc     LIBCMT:undname.obj
 0001:00001a00       ??_C@_02FODMEDOG@?$DM?$DM?$AA@ 10002a00     LIBCMT:undname.obj
 0001:00001a04       ??_C@_02GPIOPFAK@?$DO?$DO?$AA@ 10002a04     LIBCMT:undname.obj
 0001:00001a08       ??_C@_01NEMOKFLO@?$DN?$AA@ 10002a08     LIBCMT:undname.obj
 0001:00001a0c       ??_C@_07FPCDHGMM@?5delete?$AA@ 10002a0c     LIBCMT:undname.obj
 0001:00001a14       ??_C@_04NIHEBCM@?5new?$AA@ 10002a14     LIBCMT:undname.obj
 0001:00001a19       ??_C@_00CNPNBAHC@?$AA@     10002a19     LIBCMT:undname.obj
 0001:00001a1c       ??_C@_0M@GFIIJFMG@__unaligned?$AA@ 10002a1c     LIBCMT:undname.obj
 0001:00001a28       ??_C@_0L@PILCLIHE@__restrict?$AA@ 10002a28     LIBCMT:undname.obj
 0001:00001a34       ??_C@_07JOMMBBKO@__ptr64?$AA@ 10002a34     LIBCMT:undname.obj
 0001:00001a3c       ??_C@_06GHPCKEAG@__eabi?$AA@ 10002a3c     LIBCMT:undname.obj
 0001:00001a44       ??_C@_09HIJEGCPM@__clrcall?$AA@ 10002a44     LIBCMT:undname.obj
 0001:00001a50       ??_C@_0L@JMKHOMEK@__fastcall?$AA@ 10002a50     LIBCMT:undname.obj
 0001:00001a5c       ??_C@_0L@NPHFGOKO@__thiscall?$AA@ 10002a5c     LIBCMT:undname.obj
 0001:00001a68       ??_C@_09IFJBGAPI@__stdcall?$AA@ 10002a68     LIBCMT:undname.obj
 0001:00001a74       ??_C@_08GHMPAG@__pascal?$AA@ 10002a74     LIBCMT:undname.obj
 0001:00001a80       ??_C@_07KOLFKCDI@__cdecl?$AA@ 10002a80     LIBCMT:undname.obj
 0001:00001a88       ??_C@_08EHJDFFNH@__based?$CI?$AA@ 10002a88     LIBCMT:undname.obj
 0001:00001c1c       ??_C@_0BI@DFKBFLJE@GetProcessWindowStation?$AA@ 10002c1c     LIBCMT:crtmboxw.obj
 0001:00001c34       ??_C@_0BK@DEKFELLI@GetUserObjectInformationW?$AA@ 10002c34     LIBCMT:crtmboxw.obj
 0001:00001c50       ??_C@_0BD@HHGDFDBJ@GetLastActivePopup?$AA@ 10002c50     LIBCMT:crtmboxw.obj
 0001:00001c64       ??_C@_0BA@HNOPNCHB@GetActiveWindow?$AA@ 10002c64     LIBCMT:crtmboxw.obj
 0001:00001c74       ??_C@_0M@DLDCCGNP@MessageBoxW?$AA@ 10002c74     LIBCMT:crtmboxw.obj
 0001:00001c80       ??_C@_1BG@GOEBHBDC@?$AAU?$AAS?$AAE?$AAR?$AA3?$AA2?$AA?4?$AAD?$AAL?$AAL?$AA?$AA@ 10002c80     LIBCMT:crtmboxw.obj
 0001:00001ca0       ___newctype                10002ca0     LIBCMT:ctype.obj
 0001:00001fa0       __wctype                   10002fa0     LIBCMT:ctype.obj
 0001:000021a8       ___newclmap                100031a8     LIBCMT:ctype.obj
 0001:00002328       ___newcumap                10003328     LIBCMT:ctype.obj
 0001:00002528       ??_7_com_error@@6B@        10003528     comsuppw:comraise.obj
 0001:0000252c       __FPinit                   1000352c     LIBCMT:_fpinit_.obj
 0001:00002530       ??_C@_05KLBDPFGC@e?$CL000?$AA@ 10003530     LIBCMT:cvt.obj
 0001:00002538       ??_C@_06IMKFLFPG@1?$CDQNAN?$AA@ 10003538     LIBCMT:_x10fout_.obj
 0001:00002540       ??_C@_05DNEBIAHO@1?$CDINF?$AA@ 10003540     LIBCMT:_x10fout_.obj
 0001:00002548       ??_C@_05PHHOCPM@1?$CDIND?$AA@ 10003548     LIBCMT:_x10fout_.obj
 0001:00002550       ??_C@_06PGGFOGJG@1?$CDSNAN?$AA@ 10003550     LIBCMT:_x10fout_.obj
 0001:00002558       __load_config_used         10003558     LIBCMT:loadcfg.obj
 0001:000025a0       ??_R4bad_alloc@std@@6B@    100035a0     LIBCMT:new.obj
 0001:000025b4       ??_R3bad_alloc@std@@8      100035b4     LIBCMT:new.obj
 0001:000025c4       ??_R2bad_alloc@std@@8      100035c4     LIBCMT:new.obj
 0001:000025d0       ??_R1A@?0A@EA@bad_alloc@std@@8 100035d0     LIBCMT:new.obj
 0001:000025ec       ??_R1A@?0A@EA@exception@std@@8 100035ec     LIBCMT:new.obj
 0001:00002608       ??_R3exception@std@@8      10003608     LIBCMT:new.obj
 0001:00002618       ??_R2exception@std@@8      10003618     LIBCMT:new.obj
 0001:00002620       ??_R4exception@std@@6B@    10003620     LIBCMT:stdexcpt.obj
 0001:00002634       ??_R4type_info@@6B@        10003634     LIBCMT:typinfo.obj
 0001:00002648       ??_R3type_info@@8          10003648     LIBCMT:typinfo.obj
 0001:00002658       ??_R2type_info@@8          10003658     LIBCMT:typinfo.obj
 0001:00002660       ??_R1A@?0A@EA@type_info@@8 10003660     LIBCMT:typinfo.obj
 0001:00002680       ___safe_se_handler_table   10003680     <linker-defined>
 0001:00002690       ___rtc_iaa                 10003690     LIBCMT:_initsect_.obj
 0001:00002694       ___rtc_izz                 10003694     LIBCMT:_initsect_.obj
 0001:00002698       ___rtc_taa                 10003698     LIBCMT:_initsect_.obj
 0001:0000269c       ___rtc_tzz                 1000369c     LIBCMT:_initsect_.obj
 0001:000026a0       __chkstk                   100036a0 f   chkstk.obj
 0001:000026a0       __alloca_probe             100036a0     chkstk.obj
 0001:000026d0       _GetGlobalInfoW@4          100036d0 f   EMenu.obj
 0001:00002750       _SetStartupInfoW@4         10003750 f   EMenu.obj
 0001:00002790       _GetPluginInfoW@4          10003790 f   EMenu.obj
 0001:000027a0       _OpenW@4                   100037a0 f   EMenu.obj
 0001:000027c0       _ConfigureW@4              100037c0 f   EMenu.obj
 0001:000027d0       _ExitFARW@4                100037d0 f   EMenu.obj
 0001:00002800       ??0auto_sz@@QAE@XZ         10003800 f   auto_sz.obj
 0001:00002810       ??Bauto_sz@@QAEPA_WXZ      10003810 f   auto_sz.obj
 0001:00002810       ??Bauto_sz@@QAEPB_WXZ      10003810 f   auto_sz.obj
 0001:00002820       ??Aauto_sz@@QAE_WH@Z       10003820 f   auto_sz.obj
 0001:00002830       ?Realloc@auto_sz@@QAEXI@Z  10003830 f   auto_sz.obj
 0001:000028d0       ??Yauto_sz@@QAEAAV0@PB_W@Z 100038d0 f   auto_sz.obj
 0001:00002910       ?Len@auto_sz@@QBEIXZ       10003910 f   auto_sz.obj
 0001:00002920       ?Trunc@auto_sz@@QAEXI@Z    10003920 f   auto_sz.obj
 0001:00002940       ??9auto_sz@@QAE_NPB_W@Z    10003940 f   auto_sz.obj
 0001:00002960       ?CompareExcluding@auto_sz@@QAE_NPB_W_W@Z 10003960 f   auto_sz.obj
 0001:000029c0       ?RemoveTrailing@auto_sz@@QAEX_W@Z 100039c0 f   auto_sz.obj
 0001:00002a00       ?IsEmpty@auto_sz@@QAE_NXZ  10003a00 f   auto_sz.obj
 0001:00002a20       ??0auto_sz@@QAE@PB_WI@Z    10003a20 f   auto_sz.obj
 0001:00002a50       ??1auto_sz@@QAE@XZ         10003a50 f   auto_sz.obj
 0001:00002a80       ??4auto_sz@@QAEAAV0@PB_W@Z 10003a80 f   auto_sz.obj
 0001:00002af0       ??4auto_sz@@QAEAAV0@ABV0@@Z 10003af0 f   auto_sz.obj
 0001:00002b20       ??0auto_sz@@QAE@PB_W@Z     10003b20 f   auto_sz.obj
 0001:00002b40       ??0auto_sz@@QAE@ABU_STRRET@@PBU_ITEMIDLIST@@@Z 10003b40 f   auto_sz.obj
 0001:00002bc0       ??0CFarMenu@@QAE@PB_WPBU_GUID@@I@Z 10003bc0 f   FarMenu.obj
 0001:00002c50       ??1CFarMenu@@QAE@XZ        10003c50 f   FarMenu.obj
 0001:00002cb0       ?InsertItem@CFarMenu@@QAEIIPB_W_NW4ECheck@1@1@Z 10003cb0 f   FarMenu.obj
 0001:00002df0       ?AddArrows@CFarMenu@@IAEXXZ 10003df0 f   FarMenu.obj
 0001:00002f70       ??ACFarMenu@@QAEPB_WI@Z    10003f70 f   FarMenu.obj
 0001:00002fb0       ?GetCursorXY@CFarMenu@@QAEXPAH0@Z 10003fb0 f   FarMenu.obj
 0001:00003090       ?Show@CFarMenu@@QAEHPB_WH_N@Z 10004090 f   FarMenu.obj
 0001:000032c0       ?AddItem@CFarMenu@@QAEIPB_W_NW4ECheck@1@1@Z 100042c0 f   FarMenu.obj
 0001:000032e0       ?AddSeparator@CFarMenu@@QAEXXZ 100042e0 f   FarMenu.obj
 0001:00003370       ?MenuDlgProc@@YGHPAUHWND__@@IIJ@Z 10004370 f   MenuDlg.obj
 0001:00003530       ?ThreadProc@OleThread@@YGKPAX@Z 10004530 f   OleThread.obj
 0001:00003640       ?EnsureThreadStarted@OleThread@@YA_NXZ 10004640 f   OleThread.obj
 0001:00003770       ?OpenPlugin@OleThread@@YA?AW4EDoMenu@CPlugin@@HH@Z 10004770 f   OleThread.obj
 0001:00003830       ?ShowMenu@OleThread@@YAHAAVCFarMenu@@PB_WH_N@Z 10004830 f   OleThread.obj
 0001:00003890       ?Stop@OleThread@@YAXXZ     10004890 f   OleThread.obj
 0001:000038b0       ?Startup@OleThread@@YAXXZ  100048b0 f   OleThread.obj
 0001:00003970       ?Cleanup@OleThread@@YAXXZ  10004970 f   OleThread.obj
 0001:00003a50       ??0CPidl@@QAE@XZ           10004a50 f   Pidl.obj
 0001:00003a60       ??1CPidl@@QAE@XZ           10004a60 f   Pidl.obj
 0001:00003a90       ??BCPidl@@QAEPAU_ITEMIDLIST@@XZ 10004a90 f   Pidl.obj
 0001:00003aa0       ?EnsureSpace@CPidl@@QAEXXZ 10004aa0 f   Pidl.obj
 0001:00003af0       ??ICPidl@@QAEPAPAU_ITEMIDLIST@@XZ 10004af0 f   Pidl.obj
 0001:00003af0       ?GetArray@CPidl@@QAEPAPBU_ITEMIDLIST@@XZ 10004af0 f   Pidl.obj
 0001:00003b10       ?Insert@CPidl@@QAEXIPAU_ITEMIDLIST@@@Z 10004b10 f   Pidl.obj
 0001:00003ba0       ?GetAt@CPidl@@QAEPAU_ITEMIDLIST@@I@Z 10004ba0 f   Pidl.obj
 0001:00003bc0       ?Count@CPidl@@QAEIXZ       10004bc0 f   Pidl.obj
 0001:00003bd0       ?Add@CPidl@@QAEXPAU_ITEMIDLIST@@@Z 10004bd0 f   Pidl.obj
 0001:00003bf0       ?GetLangString@PluginDialogBuilder@@MAEPB_WH@Z 10004bf0 f i Plugin.obj
 0001:00003c10       ?IsWindowsVersionOrGreater@@YA_NGGG@Z 10004c10 f i Plugin.obj
 0001:00003cc0       ??1CPlugin@@QAE@XZ         10004cc0 f   Plugin.obj
 0001:00003cd0       ?ReadRegValues@CPlugin@@IAEXXZ 10004cd0 f   Plugin.obj
 0001:00003fd0       ?Message@CPlugin@@IAEHKPB_WPBQB_WHH@Z 10004fd0 f   Plugin.obj
 0001:00004010       ?CfgDlgProc@CPlugin@@IAEXPAXHH0@Z 10005010 f   Plugin.obj
 0001:000040e0       ?ExitFAR@CPlugin@@QAEXXZ   100050e0 f   Plugin.obj
 0001:000040f0       ?OpenPlugin@CPlugin@@QAEPAXHH@Z 100050f0 f   Plugin.obj
 0001:00004280       ?ParseParams@CPlugin@@IAEIPA_WPAPB_W@Z 10005280 f   Plugin.obj
 0001:00004320       ?GetFilesFromPanel@CPlugin@@IAE_NPAPAPB_WPAI1PAVauto_sz@@@Z 10005320 f   Plugin.obj
 0001:000046c0       ?ShowGuiMenu@CPlugin@@IAE_NPAUHMENU__@@PAUIContextMenu@@PAUIContextMenu2@@PAUIContextMenu3@@PAH@Z 100056c0 f   Plugin.obj
 0001:000047f0       ?GetAdditionalString@CPlugin@@IAE_NPAUIContextMenu@@IW4EAdditionalStr@1@PAVauto_sz@@@Z 100057f0 f   Plugin.obj
 0001:000048e0       ?SaveValue@?$DialogItemBinding@UFarDialogItem@@@@UAEXPAUFarDialogItem@@H@Z 100058e0 f i Plugin.obj
 0001:000048e0       ?InitDialogItem@?$DialogBuilderBase@UFarDialogItem@@@@MAEXPAUFarDialogItem@@PB_W@Z 100058e0 f i Plugin.obj
 0001:000048f0       ?TextWidth@?$DialogBuilderBase@UFarDialogItem@@@@MAEHABUFarDialogItem@@@Z 100058f0 f i Plugin.obj
 0001:00004900       ?CreateRadioButtonBinding@?$DialogBuilderBase@UFarDialogItem@@@@MAEPAU?$DialogItemBinding@UFarDialogItem@@@@PAH@Z 10005900 f i Plugin.obj
 0001:00004900       ?GetLangString@?$DialogBuilderBase@UFarDialogItem@@@@MAEPB_WH@Z 10005900 f i Plugin.obj
 0001:00004910       ?DoShowDialog@?$DialogBuilderBase@UFarDialogItem@@@@MAEHXZ 10005910 f i Plugin.obj
 0001:00004920       ??1?$DialogBuilderBase@UFarDialogItem@@@@MAE@XZ 10005920 f i Plugin.obj
 0001:00004970       ?AddIntEditField@?$DialogBuilderBase@UFarDialogItem@@@@UAEPAUFarDialogItem@@PAHH@Z 10005970 f i Plugin.obj
 0001:00004970       ?CreateCheckBoxBinding@?$DialogBuilderBase@UFarDialogItem@@@@MAEPAU?$DialogItemBinding@UFarDialogItem@@@@PAHH@Z 10005970 f i Plugin.obj
 0001:00004970       ?AddUIntEditField@?$DialogBuilderBase@UFarDialogItem@@@@UAEPAUFarDialogItem@@PAIH@Z 10005970 f i Plugin.obj
 0001:00004980       ??_E?$DialogBuilderBase@UFarDialogItem@@@@MAEPAXI@Z 10005980 f i Plugin.obj
 0001:00004980       ??_G?$DialogBuilderBase@UFarDialogItem@@@@MAEPAXI@Z 10005980 f i Plugin.obj
 0001:000049a0       ?ReallocDialogItems@?$DialogBuilderBase@UFarDialogItem@@@@IAEXXZ 100059a0 f i Plugin.obj
 0001:00004a70       ?UpdateSecondColumnPosition@?$DialogBuilderBase@UFarDialogItem@@@@IAEXXZ 10005a70 f i Plugin.obj
 0001:00004ad0       ?SaveValues@?$DialogBuilderBase@UFarDialogItem@@@@IAEXXZ 10005ad0 f i Plugin.obj
 0001:00004b20       ?MaxTextWidth@?$DialogBuilderBase@UFarDialogItem@@@@IAEHXZ 10005b20 f i Plugin.obj
 0001:00004be0       ??1CHMenu@@QAE@XZ          10005be0 f i Plugin.obj
 0001:00004c00       ?InitDialogItem@PluginDialogBuilder@@MAEXPAUFarDialogItem@@PB_W@Z 10005c00 f i Plugin.obj
 0001:00004c20       ?TextWidth@PluginDialogBuilder@@MAEHABUFarDialogItem@@@Z 10005c20 f i Plugin.obj
 0001:00004c40       ?DoShowDialog@PluginDialogBuilder@@MAEHXZ 10005c40 f i Plugin.obj
 0001:00004ca0       ?SaveValue@PluginCheckBoxBinding@@UAEXPAUFarDialogItem@@H@Z 10005ca0 f i Plugin.obj
 0001:00004ce0       ?SaveValue@PluginRadioButtonBinding@@UAEXPAUFarDialogItem@@H@Z 10005ce0 f i Plugin.obj
 0001:00004d10       ??0PluginIntEditFieldBinding@@QAE@ABUPluginStartupInfo@@PAPAXHPAHH@Z 10005d10 f i Plugin.obj
 0001:00004db0       ?SaveValue@PluginIntEditFieldBinding@@UAEXPAUFarDialogItem@@H@Z 10005db0 f i Plugin.obj
 0001:00004de0       ??0PluginUIntEditFieldBinding@@QAE@ABUPluginStartupInfo@@PAPAXHPAIH@Z 10005de0 f i Plugin.obj
 0001:00004e80       ?SaveValue@PluginUIntEditFieldBinding@@UAEXPAUFarDialogItem@@H@Z 10005e80 f i Plugin.obj
 0001:00004eb0       ?CreateCheckBoxBinding@PluginDialogBuilder@@MAEPAU?$DialogItemBinding@UFarDialogItem@@@@PAHH@Z 10005eb0 f i Plugin.obj
 0001:00004f00       ?CreateRadioButtonBinding@PluginDialogBuilder@@MAEPAU?$DialogItemBinding@UFarDialogItem@@@@PAH@Z 10005f00 f i Plugin.obj
 0001:00004f50       ??_GPluginDialogBuilder@@UAEPAXI@Z 10005f50 f i Plugin.obj
 0001:00004f50       ??_EPluginDialogBuilder@@UAEPAXI@Z 10005f50 f i Plugin.obj
 0001:00004fa0       ??0CPlugin@@QAE@PBUPluginStartupInfo@@@Z 10005fa0 f   Plugin.obj
 0001:00005070       ?GetPluginInfo@CPlugin@@QAEXPAUPluginInfo@@@Z 10006070 f   Plugin.obj
 0001:000050d0       ?CfgDlgProcStatic@CPlugin@@KGHPAXHH0@Z 100060d0 f   Plugin.obj
 0001:00005120       ?GetFilesFromParams@CPlugin@@IAE_NPA_WPAPAPB_WPAI2PAVauto_sz@@_N@Z 10006120 f   Plugin.obj
 0001:000052a0       ?AddCheckbox@?$DialogBuilderBase@UFarDialogItem@@@@QAEPAUFarDialogItem@@HPAHH_N@Z 100062a0 f i Plugin.obj
 0001:000053d0       ?AddRadioButtons@?$DialogBuilderBase@UFarDialogItem@@@@QAEXPAHHQBH_N@Z 100063d0 f i Plugin.obj
 0001:00005530       ?AddButtons@?$DialogBuilderBase@UFarDialogItem@@@@QAEXHPBHHH@Z 10006530 f i Plugin.obj
 0001:00005690       ?UpdateBorderSize@?$DialogBuilderBase@UFarDialogItem@@@@IAEXXZ 10006690 f i Plugin.obj
 0001:00005740       ?AddSeparator@?$DialogBuilderBase@UFarDialogItem@@@@QAEXPB_W@Z 10006740 f i Plugin.obj
 0001:000057b0       ??_EPluginUIntEditFieldBinding@@UAEPAXI@Z 100067b0 f i Plugin.obj
 0001:000057b0       ??_EPluginIntEditFieldBinding@@UAEPAXI@Z 100067b0 f i Plugin.obj
 0001:000057b0       ??_EPluginRadioButtonBinding@@UAEPAXI@Z 100067b0 f i Plugin.obj
 0001:000057b0       ??_GPluginIntEditFieldBinding@@UAEPAXI@Z 100067b0 f i Plugin.obj
 0001:000057b0       ??_EPluginCheckBoxBinding@@UAEPAXI@Z 100067b0 f i Plugin.obj
 0001:000057b0       ??_E?$DialogItemBinding@UFarDialogItem@@@@UAEPAXI@Z 100067b0 f i Plugin.obj
 0001:000057b0       ??_GPluginUIntEditFieldBinding@@UAEPAXI@Z 100067b0 f i Plugin.obj
 0001:000057b0       ??_GPluginCheckBoxBinding@@UAEPAXI@Z 100067b0 f i Plugin.obj
 0001:000057b0       ??_G?$DialogItemBinding@UFarDialogItem@@@@UAEPAXI@Z 100067b0 f i Plugin.obj
 0001:000057b0       ??_GPluginRadioButtonBinding@@UAEPAXI@Z 100067b0 f i Plugin.obj
 0001:000057d0       ??0PluginDialogBuilder@@QAE@ABUPluginStartupInfo@@ABU_GUID@@1HPB_WP6GHPAXHH3@Z3_K@Z 100067d0 f i Plugin.obj
 0001:000058e0       ?AddIntEditField@PluginDialogBuilder@@UAEPAUFarDialogItem@@PAHH@Z 100068e0 f i Plugin.obj
 0001:000059a0       ?AddUIntEditField@PluginDialogBuilder@@UAEPAUFarDialogItem@@PAIH@Z 100069a0 f i Plugin.obj
 0001:00005a60       ?ShowFolder@CPlugin@@IAE_NPAUIShellFolder@@PBU_ITEMIDLIST@@PAHPB_WPAPAUIDropTarget@@@Z 10006a60 f   Plugin.obj
 0001:00005d80       ??$_QueryInterface@V?$_com_ptr_t@V?$_com_IIID@UIContextMenu@@$1?_GUID_000214e4_0000_0000_c000_000000000046@@3U__s_GUID@@B@@@@@?$_com_ptr_t@V?$_com_IIID@UIContextMenu2@@$1?_GUID_000214f4_0000_0000_c000_000000000046@@3U__s_GUID@@B@@@@AAEJV?$_com_ptr_t@V?$_com_IIID@UIContextMenu@@$1?_GUID_000214e4_0000_0000_c000_000000000046@@3U__s_GUID@@B@@@@@Z 10006d80 f i Plugin.obj
 0001:00005e00       ??$_QueryInterface@V?$_com_ptr_t@V?$_com_IIID@UIContextMenu@@$1?_GUID_000214e4_0000_0000_c000_000000000046@@3U__s_GUID@@B@@@@@?$_com_ptr_t@V?$_com_IIID@UIContextMenu3@@$1?_GUID_bcfce0a0_ec17_11d0_8d10_00a0c90f2719@@3U__s_GUID@@B@@@@AAEJV?$_com_ptr_t@V?$_com_IIID@UIContextMenu@@$1?_GUID_000214e4_0000_0000_c000_000000000046@@3U__s_GUID@@B@@@@@Z 10006e00 f i Plugin.obj
 0001:00005e80       ?ShowTextMenu@CPlugin@@IAE_NPAUHMENU__@@PAUIContextMenu@@PAUIContextMenu2@@PAUIContextMenu3@@PAHPB_WPAUIShellFolder@@PAPBU_ITEMIDLIST@@I@Z 10006e80 f   Plugin.obj
 0001:00006400       ?Configure@CPlugin@@QAEHXZ 10007400 f   Plugin.obj
 0001:00006a20       ?DoMenu@CPlugin@@IAE?AW4EDoMenu@1@PAUIShellFolder@@PAPBU_ITEMIDLIST@@QAPB_WIIPB_WW4EAutoItem@1@@Z 10007a20 f   Plugin.obj
 0001:00007380       ?SelectDrive@CPlugin@@IAE?AW4EDoMenu@1@XZ 10008380 f   Plugin.obj
 0001:000077a0       ?MenuForPanelOrCmdLine@CPlugin@@IAE?AW4EDoMenu@1@PA_WW4EAutoItem@1@@Z 100087a0 f   Plugin.obj
 0001:00007b90       ?DoMenu@CPlugin@@IAE?AW4EDoMenu@1@PA_WW4CallMode@1@@Z 10008b90 f   Plugin.obj
 0001:00007e10       ?OpenPluginBkg@CPlugin@@QAE?AW4EDoMenu@1@HH@Z 10008e10 f   Plugin.obj
 0001:00007f37       ??1bad_alloc@std@@UAE@XZ   10008f37 f i LIBCMT:new.obj
 0001:00007f42       ??_Ebad_alloc@std@@UAEPAXI@Z 10008f42 f i LIBCMT:new.obj
 0001:00007f42       ??_Gbad_alloc@std@@UAEPAXI@Z 10008f42 f i LIBCMT:new.obj
 0001:00007f69       ??0bad_alloc@std@@QAE@ABV01@@Z 10008f69 f i LIBCMT:new.obj
 0001:00007f86       ??2@YAPAXI@Z               10008f86 f   LIBCMT:new.obj
 0001:00008006       ??3@YAXPAX@Z               10009006 f   LIBCMT:delete.obj
 0001:00008020       _memmove                   10009020 f   LIBCMT:memmove.obj
 0001:00008390       _memcpy                    10009390 f   LIBCMT:memcpy.obj
 0001:00008700       _memset                    10009700 f   LIBCMT:memset.obj
 0001:00008788       __except_handler3          10009788 f   LIBCMT:exsup3.obj
 0001:00008886       __seh_longjmp_unwind@4     10009886 f   LIBCMT:exsup3.obj
 0001:000088a1       __CRT_INIT@12              100098a1 f   LIBCMT:dllcrt0.obj
 0001:00008afb       __DllMainCRTStartup@12     10009afb f   LIBCMT:dllcrt0.obj
 0001:00008b1e       ??0exception@std@@QAE@ABQBDH@Z 10009b1e f   LIBCMT:stdexcpt.obj
 0001:00008b3b       ?what@exception@std@@UBEPBDXZ 10009b3b f   LIBCMT:stdexcpt.obj
 0001:00008b48       ?_Copy_str@exception@std@@AAEXPBD@Z 10009b48 f   LIBCMT:stdexcpt.obj
 0001:00008b88       ?_Tidy@exception@std@@AAEXXZ 10009b88 f   LIBCMT:stdexcpt.obj
 0001:00008ba6       ??4exception@std@@QAEAAV01@ABV01@@Z 10009ba6 f   LIBCMT:stdexcpt.obj
 0001:00008bdb       ??1exception@std@@UAE@XZ   10009bdb f   LIBCMT:stdexcpt.obj
 0001:00008be6       ??_Eexception@std@@UAEPAXI@Z 10009be6 f i LIBCMT:stdexcpt.obj
 0001:00008be6       ??_Gexception@std@@UAEPAXI@Z 10009be6 f i LIBCMT:stdexcpt.obj
 0001:00008c0d       ??0exception@std@@QAE@ABV01@@Z 10009c0d f   LIBCMT:stdexcpt.obj
 0001:00008c32       ??1type_info@@UAE@XZ       10009c32 f   LIBCMT:typinfo.obj
 0001:00008c42       ??_Gtype_info@@UAEPAXI@Z   10009c42 f i LIBCMT:typinfo.obj
 0001:00008c42       ??_Etype_info@@UAEPAXI@Z   10009c42 f i LIBCMT:typinfo.obj
 0001:00008d19       ___onexitinit              10009d19 f   LIBCMT:onexit.obj
 0001:00008d4a       __onexit                   10009d4a f   LIBCMT:onexit.obj
 0001:00008d86       _atexit                    10009d86 f   LIBCMT:onexit.obj
 0001:00008d9d       _malloc                    10009d9d f   LIBCMT:malloc.obj
 0001:00008e31       __initp_heap_handler       10009e31 f   LIBCMT:handler.obj
 0001:00008e40       __callnewh                 10009e40 f   LIBCMT:handler.obj
 0001:00008e68       __CxxThrowException@8      10009e68 f   LIBCMT:throw.obj
 0001:00008eb4       _free                      10009eb4 f   LIBCMT:free.obj
 0001:00008eee       __VEC_memcpy               10009eee f   LIBCMT:p4_memcpy.obj
 0001:00008ff1       ___sse2_available_init     10009ff1 f   LIBCMT:cpu_disp.obj
 0001:00009001       __VEC_memzero              1000a001 f   LIBCMT:p4_memset.obj
 0001:000090bb       _CallDestructExceptionObject 1000a0bb f   LIBCMT:calldtor.obj
 0001:00009100       __global_unwind2           1000a100 f   LIBCMT:exsup.obj
 0001:00009165       __local_unwind2            1000a165 f   LIBCMT:exsup.obj
 0001:000091e9       __abnormal_termination     1000a1e9 f   LIBCMT:exsup.obj
 0001:0000920c       __NLG_Notify1              1000a20c f   LIBCMT:exsup.obj
 0001:00009215       __NLG_Notify               1000a215 f   LIBCMT:exsup.obj
 0001:0000922c       __NLG_Dispatch             1000a22c     LIBCMT:exsup.obj
 0001:0000922c       __NLG_Dispatch2            1000a22c     LIBCMT:exsup.obj
 0001:00009234       __NLG_Call                 1000a234 f   LIBCMT:exsup.obj
 0001:00009236       __NLG_Return2              1000a236     LIBCMT:exsup.obj
 0001:00009300       __ValidateEH3RN            1000a300 f   LIBCMT:eh3valid.obj
 0001:00009646       __encoded_null             1000a646 f   LIBCMT:tidtable.obj
 0001:0000964f       ___crtTlsAlloc@4           1000a64f f   LIBCMT:tidtable.obj
 0001:00009658       ___set_flsgetvalue         1000a658 f   LIBCMT:tidtable.obj
 0001:0000968c       __mtterm                   1000a68c f   LIBCMT:tidtable.obj
 0001:000096c9       __initptd                  1000a6c9 f   LIBCMT:tidtable.obj
 0001:0000977d       __getptd_noexit            1000a77d f   LIBCMT:tidtable.obj
 0001:000097f6       __getptd                   1000a7f6 f   LIBCMT:tidtable.obj
 0001:00009810       __freefls@4                1000a810 f   LIBCMT:tidtable.obj
 0001:0000993f       __freeptd                  1000a93f f   LIBCMT:tidtable.obj
 0001:000099ad       __mtinit                   1000a9ad f   LIBCMT:tidtable.obj
 0001:00009b28       __malloc_crt               1000ab28 f   LIBCMT:crtheap.obj
 0001:00009b6d       __calloc_crt               1000ab6d f   LIBCMT:crtheap.obj
 0001:00009bb9       __realloc_crt              1000abb9 f   LIBCMT:crtheap.obj
 0001:00009c07       ___crtCorExitProcess       1000ac07 f   LIBCMT:crt0dat.obj
 0001:00009c32       ___crtExitProcess          1000ac32 f   LIBCMT:crt0dat.obj
 0001:00009c4a       __lockexit                 1000ac4a f   LIBCMT:crt0dat.obj
 0001:00009c53       __unlockexit               1000ac53 f   LIBCMT:crt0dat.obj
 0001:00009c5c       __init_pointers            1000ac5c f   LIBCMT:crt0dat.obj
 0001:00009c8f       __initterm_e               1000ac8f f   LIBCMT:crt0dat.obj
 0001:00009cb3       __cinit                    1000acb3 f   LIBCMT:crt0dat.obj
 0001:00009e8a       __exit                     1000ae8a f   LIBCMT:crt0dat.obj
 0001:00009ea0       __cexit                    1000aea0 f   LIBCMT:crt0dat.obj
 0001:00009eaf       __amsg_exit                1000aeaf f   LIBCMT:crt0dat.obj
 0001:00009ecd       __ioinit                   1000aecd f   LIBCMT:ioinit.obj
 0001:0000a112       __ioterm                   1000b112 f   LIBCMT:ioinit.obj
 0001:0000a165       __setenvp                  1000b165 f   LIBCMT:stdenvp.obj
 0001:0000a3db       __setargv                  1000b3db f   LIBCMT:stdargv.obj
 0001:0000a496       ___crtGetEnvironmentStringsA 1000b496 f   LIBCMT:a_env.obj
 0001:0000a52d       __RTC_Initialize           1000b52d f   LIBCMT:_initsect_.obj
 0001:0000a553       __RTC_Terminate            1000b553 f   LIBCMT:_initsect_.obj
 0001:0000a579       __heap_init                1000b579 f   LIBCMT:heapinit.obj
 0001:0000a597       __heap_term                1000b597 f   LIBCMT:heapinit.obj
 0001:0000a5b0       __SEH_prolog4              1000b5b0 f   LIBCMT:sehprolg4.obj
 0001:0000a5f5       __SEH_epilog4              1000b5f5 f   LIBCMT:sehprolg4.obj
 0001:0000a610       __except_handler4          1000b610 f   LIBCMT:chandler4.obj
 0001:0000a79f       __XcptFilter               1000b79f f   LIBCMT:winxfltr.obj
 0001:0000a8e9       ___CppXcptFilter           1000b8e9 f   LIBCMT:winxfltr.obj
 0001:0000a909       _DllMain@12                1000b909 f   LIBCMT:dllmain.obj
 0001:0000a90f       ___security_init_cookie    1000b90f f   LIBCMT:gs_support.obj
 0001:0000a9aa       _strcpy_s                  1000b9aa f   LIBCMT:strcpy_s.obj
 0001:0000aa10       _strlen                    1000ba10 f   LIBCMT:strlen.obj
 0001:0000aa9b       ?_Type_info_dtor@type_info@@CAXPAV1@@Z 1000ba9b f   LIBCMT:typname.obj
 0001:0000ab10       _strcmp                    1000bb10 f   LIBCMT:strcmp.obj
 0001:0000ab98       __msize                    1000bb98 f   LIBCMT:msize.obj
 0001:0000abcb       __GET_RTERRMSG             1000bbcb f   LIBCMT:crt0msg.obj
 0001:0000abf1       __NMSG_WRITE               1000bbf1 f   LIBCMT:crt0msg.obj
 0001:0000ada0       __FF_MSGBANNER             1000bda0 f   LIBCMT:crt0msg.obj
 0001:0000add9       __get_errno_from_oserr     1000bdd9 f   LIBCMT:dosmap.obj
 0001:0000ae1b       __errno                    1000be1b f   LIBCMT:dosmap.obj
 0001:0000ae2e       __mtinitlocks              1000be2e f   LIBCMT:mlock.obj
 0001:0000ae78       __mtdeletelocks            1000be78 f   LIBCMT:mlock.obj
 0001:0000aecf       __unlock                   1000becf f   LIBCMT:mlock.obj
 0001:0000aee6       __mtinitlocknum            1000bee6 f   LIBCMT:mlock.obj
 0001:0000afa8       __lock                     1000bfa8 f   LIBCMT:mlock.obj
 0001:0000afe0       __ValidateImageBase        1000bfe0 f   LIBCMT:pesect.obj
 0001:0000b020       __FindPESection            1000c020 f   LIBCMT:pesect.obj
 0001:0000b070       __IsNonwritableInCurrentImage 1000c070 f   LIBCMT:pesect.obj
 0001:0000b12c       @__security_check_cookie@4 1000c12c f   LIBCMT:secchk.obj
 0001:0000b13b       ___addlocaleref            1000c13b f   LIBCMT:localref.obj
 0001:0000b1ca       ___removelocaleref         1000c1ca f   LIBCMT:localref.obj
 0001:0000b263       ___freetlocinfo            1000c263 f   LIBCMT:localref.obj
 0001:0000b3ae       __updatetlocinfoEx_nolock  1000c3ae f   LIBCMT:localref.obj
 0001:0000b3fb       ___updatetlocinfo          1000c3fb f   LIBCMT:localref.obj
 0001:0000b697       ___updatetmbcinfo          1000c697 f   LIBCMT:mbctype.obj
 0001:0000b73b       ??0_LocaleUpdate@@QAE@PAUlocaleinfo_struct@@@Z 1000c73b f i LIBCMT:mbctype.obj
 0001:0000b83e       __setmbcp_nolock           1000c83e f   LIBCMT:mbctype.obj
 0001:0000ba27       __setmbcp                  1000ca27 f   LIBCMT:mbctype.obj
 0001:0000bbc1       ___initmbctable            1000cbc1 f   LIBCMT:mbctype.obj
 0001:0000bbdf       __calloc_impl              1000cbdf f   LIBCMT:calloc_impl.obj
 0001:0000bc61       _realloc                   1000cc61 f   LIBCMT:realloc.obj
 0001:0000bd0e       ?terminate@@YAXXZ          1000cd0e f   LIBCMT:hooks.obj
 0001:0000bd47       __initp_eh_hooks           1000cd47 f   LIBCMT:hooks.obj
 0001:0000bd58       __initp_misc_winsig        1000cd58 f   LIBCMT:winsig.obj
 0001:0000bdad       ___get_sigabrt             1000cdad f   LIBCMT:winsig.obj
 0001:0000bdba       _raise                     1000cdba f   LIBCMT:winsig.obj
 0001:0000bf5d       __initp_misc_rand_s        1000cf5d f   LIBCMT:rand_s.obj
 0001:0000bf6c       __initp_misc_purevirt      1000cf6c f   LIBCMT:inithelp.obj
 0001:0000bf7b       __initp_misc_invarg        1000cf7b f   LIBCMT:invarg.obj
 0001:0000bf8a       __call_reportfault         1000cf8a f   LIBCMT:invarg.obj
 0001:0000c0b3       __invoke_watson            1000d0b3 f   LIBCMT:invarg.obj
 0001:0000c0d8       __invalid_parameter        1000d0d8 f   LIBCMT:invarg.obj
 0001:0000c105       __invalid_parameter_noinfo 1000d105 f   LIBCMT:invarg.obj
 0001:0000c115       __initp_misc_cfltcvt_tab   1000d115 f   LIBCMT:cmiscdat.obj
 0001:0000c18b       __ismbblead                1000d18b f   LIBCMT:ismbbyte.obj
 0001:0000c1b0       __local_unwind4            1000d1b0 f   LIBCMT:exsup4.obj
 0001:0000c286       __seh_longjmp_unwind4@4    1000d286 f   LIBCMT:exsup4.obj
 0001:0000c2a2       @_EH4_CallFilterFunc@8     1000d2a2 f   LIBCMT:exsup4.obj
 0001:0000c2b9       @_EH4_TransferToHandler@8  1000d2b9 f   LIBCMT:exsup4.obj
 0001:0000c2d2       @_EH4_GlobalUnwind2@8      1000d2d2 f   LIBCMT:exsup4.obj
 0001:0000c2eb       @_EH4_LocalUnwind@16       1000d2eb f   LIBCMT:exsup4.obj
 0001:0000c302       ___crtMessageBoxW          1000d302 f   LIBCMT:crtmboxw.obj
 0001:0000c46e       _wcscat_s                  1000d46e f   LIBCMT:wcscat_s.obj
 0001:0000c4e3       _wcsncpy_s                 1000d4e3 f   LIBCMT:wcsncpy_s.obj
 0001:0000c5b0       _wcslen                    1000d5b0 f   LIBCMT:wcslen.obj
 0001:0000c5cb       _wcscpy_s                  1000d5cb f   LIBCMT:wcscpy_s.obj
 0001:0000c62e       __set_error_mode           1000d62e f   LIBCMT:errmode.obj
 0001:0000c66d       ___report_gsfailure        1000d66d f   LIBCMT:gs_report.obj
 0001:0000c773       ___free_lc_time            1000d773 f   LIBCMT:inittime.obj
 0001:0000caea       ___free_lconv_num          1000daea f   LIBCMT:initnum.obj
 0001:0000cb53       ___free_lconv_mon          1000db53 f   LIBCMT:initmon.obj
 0001:0000cc51       __freea                    1000dc51 f i LIBCMT:a_map.obj
 0001:0000ce58       ___crtLCMapStringA         1000de58 f   LIBCMT:a_map.obj
 0001:0000cf85       ___crtGetStringTypeA       1000df85 f   LIBCMT:a_str.obj
 0001:0000cfc5       _abort                     1000dfc5 f   LIBCMT:abort.obj
 0001:0000cff8       __crt_debugger_hook        1000dff8 f   LIBCMT:dbghook.obj
 0001:0000d000       __fptrap                   1000e000 f   LIBCMT:crt0fp.obj
 0001:0000d010       __aulldvrm                 1000e010 f   LIBCMT:ulldvrm.obj
 0001:0000d0b0       __alloca_probe_16          1000e0b0 f   LIBCMT:alloca16.obj
 0001:0000d0c6       __alloca_probe_8           1000e0c6     LIBCMT:alloca16.obj
 0001:0000d0dc       __isctype_l                1000e0dc f   LIBCMT:isctype.obj
 0001:0000d1a0       __allmul                   1000e1a0 f   LIBCMT:llmul.obj
 0001:0000d1d4       __isleadbyte_l             1000e1d4 f i LIBCMT:_wctype.obj
 0001:0000d210       _strcspn                   1000e210 f   LIBCMT:strcspn.obj
 0001:0000d260       _strpbrk                   1000e260 f   LIBCMT:strpbrk.obj
 0001:0000d2a0       __tolower_l                1000e2a0 f   LIBCMT:tolower.obj
 0001:0000d3b5       _tolower                   1000e3b5 f   LIBCMT:tolower.obj
 0001:0000d3f0       ___ascii_strnicmp          1000e3f0 f   LIBCMT:_strnicm.obj
 0001:0000d460       ?_com_issue_error@@YGXJ@Z  1000e460 f   comsuppw:comsupp.obj
 0001:0000d480       ??1_com_error@@UAE@XZ      1000e480 f i comsuppw:comraise.obj
 0001:0000d4b0       ?_com_raise_error@@YGXJPAUIErrorInfo@@@Z 1000e4b0 f   comsuppw:comraise.obj
 0001:0000d4f0       ??0_com_error@@QAE@ABV0@@Z 1000e4f0 f i comsuppw:comraise.obj
 0001:0000d530       ??_E_com_error@@UAEPAXI@Z  1000e530 f i comsuppw:comraise.obj
 0001:0000d530       ??_G_com_error@@UAEPAXI@Z  1000e530 f i comsuppw:comraise.obj
 0001:0000d572       _RtlUnwind@16              1000e572 f   kernel32:KERNEL32.dll
 0001:0000d578       __cfltcvt_init             1000e578 f   LIBCMT:_fpinit_.obj
 0001:0000d5d8       __fpmath                   1000e5d8 f   LIBCMT:_fpinit_.obj
 0001:0000d5f1       __forcdecpt_l              1000e5f1 f   LIBCMT:cvt.obj
 0001:0000d665       __cropzeros_l              1000e665 f   LIBCMT:cvt.obj
 0001:0000d6e7       __positive                 1000e6e7 f   LIBCMT:cvt.obj
 0001:0000d703       __fassign_l                1000e703 f   LIBCMT:cvt.obj
 0001:0000d745       __fassign                  1000e745 f   LIBCMT:cvt.obj
 0001:0000d77e       __forcdecpt                1000e77e f   LIBCMT:cvt.obj
 0001:0000d791       __cropzeros                1000e791 f   LIBCMT:cvt.obj
 0001:0000d905       __cftoe_l                  1000e905 f   LIBCMT:cvt.obj
 0001:0000d9cc       __cftoe                    1000e9cc f   LIBCMT:cvt.obj
 0001:0000d9ec       __cftoa_l                  1000e9ec f   LIBCMT:cvt.obj
 0001:0000de65       __cftof_l                  1000ee65 f   LIBCMT:cvt.obj
 0001:0000df26       __cftog_l                  1000ef26 f   LIBCMT:cvt.obj
 0001:0000e013       __cfltcvt_l                1000f013 f   LIBCMT:cvt.obj
 0001:0000e09b       __cfltcvt                  1000f09b f   LIBCMT:cvt.obj
 0001:0000e0be       __setdefaultprecision      1000f0be f   LIBCMT:fp8.obj
 0001:0000e0f0       _strrchr                   1000f0f0 f   LIBCMT:strrchr.obj
 0001:0000e11d       __isdigit_l                1000f11d f i LIBCMT:_ctype.obj
 0001:0000e16e       _isdigit                   1000f16e f i LIBCMT:_ctype.obj
 0001:0000e19c       __atodbl_l                 1000f19c f   LIBCMT:atodbl.obj
 0001:0000e244       __atoflt_l                 1000f244 f   LIBCMT:atodbl.obj
 0001:0000e2ec       __fptostr                  1000f2ec f   LIBCMT:_fptostr.obj
 0001:0000e39f       ___dtold                   1000f39f f   LIBCMT:_cfout_.obj
 0001:0000e452       __fltout2                  1000f452 f   LIBCMT:_cfout_.obj
 0001:0000e4e0       __alldvrm                  1000f4e0 f   LIBCMT:lldvrm.obj
 0001:0000e5c0       __aullshr                  1000f5c0 f   LIBCMT:ullshr.obj
 0001:0000e5df       __controlfp_s              1000f5df f   LIBCMT:_contrlfp_.obj
 0001:0000e63e       __ld12tod                  1000f63e f   LIBCMT:_intrncvt_.obj
 0001:0000eb8f       __ld12tof                  1000fb8f f   LIBCMT:_intrncvt_.obj
 0001:0000f0e0       ___strgtold12_l            100100e0 f   LIBCMT:_strgtold_.obj
 0001:0000f7bc       _$I10_OUTPUT               100107bc f   LIBCMT:_x10fout_.obj
 0001:000101e2       __control87                100111e2 f i LIBCMT:_ieee87_.obj
 0001:000104f4       ___mtold12                 100114f4 f   LIBCMT:_mantold_.obj
 0001:000106d8       ___set_fpsr_sse2           100116d8 f   LIBCMT:_fpctrl_.obj
 0001:0001076c       __TI2?AVbad_alloc@std@@    1001176c     LIBCMT:new.obj
 0001:0001077c       __CTA2?AVbad_alloc@std@@   1001177c     LIBCMT:new.obj
 0001:00010788       __CT??_R0?AVbad_alloc@std@@@8??0bad_alloc@std@@QAE@ABV01@@Z12 10011788     LIBCMT:new.obj
 0001:000107a4       __CT??_R0?AVexception@std@@@8??0exception@std@@QAE@ABV01@@Z12 100117a4     LIBCMT:new.obj
 0001:000109ac       __TI1?AV_com_error@@       100119ac     comsuppw:comraise.obj
 0001:000109bc       __CTA1?AV_com_error@@      100119bc     comsuppw:comraise.obj
 0001:000109c4       __CT??_R0?AV_com_error@@@8??0_com_error@@QAE@ABV0@@Z16 100119c4     comsuppw:comraise.obj
 0001:000109fc       __IMPORT_DESCRIPTOR_KERNEL32 100119fc     kernel32:KERNEL32.dll
 0001:00010a10       __IMPORT_DESCRIPTOR_USER32 10011a10     user32:USER32.dll
 0001:00010a24       __IMPORT_DESCRIPTOR_SHELL32 10011a24     shell32:SHELL32.dll
 0001:00010a38       __IMPORT_DESCRIPTOR_ole32  10011a38     ole32:ole32.dll
 0001:00010a4c       __NULL_IMPORT_DESCRIPTOR   10011a4c     kernel32:KERNEL32.dll
 0002:00000000       ?g_szTopicMain@@3PB_WB     10013000     Plugin.obj
 0002:00000004       ?g_szTopicConfig@@3PB_WB   10013004     Plugin.obj
 0002:00000008       ?g_szTopicChooseMenuType@@3PB_WB 10013008     Plugin.obj
 0002:0000000c       ?g_szTopicContextMenu@@3PB_WB 1001300c     Plugin.obj
 0002:00000010       ?g_szTopicMyComp@@3PB_WB   10013010     Plugin.obj
 0002:00000014       ?g_szTopicError0@@3PB_WB   10013014     Plugin.obj
 0002:00000018       ?g_szTopicError1@@3PB_WB   10013018     Plugin.obj
 0002:0000001c       ?g_szTopicError2@@3PB_WB   1001301c     Plugin.obj
 0002:00000020       ?g_szTopicClose@@3PB_WB    10013020     Plugin.obj
 0002:00000024       ??_R0?AVbad_alloc@std@@@8  10013024     LIBCMT:new.obj
 0002:00000040       ??_R0?AVexception@std@@@8  10013040     LIBCMT:new.obj
 0002:00000060       ??_R0?AVtype_info@@@8      10013060     LIBCMT:typinfo.obj
 0002:00000080       __NLG_Destination          10013080     LIBCMT:exsup.obj
 0002:00000090       ___flsindex                10013090     LIBCMT:tidtable.obj
 0002:00000094       ___getvalueindex           10013094     LIBCMT:tidtable.obj
 0002:00000098       ___badioinfo               10013098     LIBCMT:ioinit.obj
 0002:00000370       ___security_cookie         10013370     LIBCMT:gs_cookie.obj
 0002:00000374       ___security_cookie_complement 10013374     LIBCMT:gs_cookie.obj
 0002:00000378       ___clocalestr              10013378     LIBCMT:nlsdata2.obj
 0002:00000380       ___lc_time_c               10013380     LIBCMT:nlsdata2.obj
 0002:000004e8       ___initiallocinfo          100134e8     LIBCMT:nlsdata2.obj
 0002:000005c0       ___ptlocinfo               100135c0     LIBCMT:nlsdata2.obj
 0002:000005c8       ___initialmbcinfo          100135c8     LIBCMT:mbctype.obj
 0002:000007e8       __mbctype                  100137e8     LIBCMT:mbctype.obj
 0002:000008f0       __mbcasemap                100138f0     LIBCMT:mbctype.obj
 0002:000009f0       ___ptmbcinfo               100139f0     LIBCMT:mbctype.obj
 0002:00000ae8       __cfltcvt_tab              10013ae8     LIBCMT:cmiscdat.obj
 0002:00000b10       ___lconv_static_decimal    10013b10     LIBCMT:lconv.obj
 0002:00000b14       ___lconv_static_W_decimal  10013b14     LIBCMT:lconv.obj
 0002:00000b18       ___lconv_c                 10013b18     LIBCMT:lconv.obj
 0002:00000b68       ___lconv                   10013b68     LIBCMT:lconv.obj
 0002:00000b6c       ___globallocalestatus      10013b6c     LIBCMT:glstatus.obj
 0002:00000b70       __pctype                   10013b70     LIBCMT:ctype.obj
 0002:00000b74       __pwctype                  10013b74     LIBCMT:ctype.obj
 0002:00000b78       ___abort_behavior          10013b78     LIBCMT:abort.obj
 0002:00000b90       ___mb_cur_max              10013b90     LIBCMT:nlsdata1.obj
 0002:00000b94       ___decimal_point           10013b94     LIBCMT:nlsdata1.obj
 0002:00000b98       ___decimal_point_length    10013b98     LIBCMT:nlsdata1.obj
 0002:00000ba0       ?__errorPfn@@3P6GXJPAUIErrorInfo@@@ZA 10013ba0     comsuppw:comsupp.obj
 0002:00000ba4       ??_R0?AV_com_error@@@8     10013ba4     comsuppw:comraise.obj
 0002:00000bc0       __fltused                  10013bc0     LIBCMT:_fpinit_.obj
 0002:00000bc4       __ldused                   10013bc4     LIBCMT:_fpinit_.obj
 0002:00000c00       __pow10pos                 10013c00     LIBCMT:_constpow_.obj
 0002:00000d60       __pow10neg                 10013d60     LIBCMT:_constpow_.obj
 0002:00000ee0       ?thePlug@@3PAVCPlugin@@A   10013ee0     EMenu.obj
 0002:00000ee4       ?Res@ShowMenuArgs@OleThread@@3HA 10013ee4     OleThread.obj
 0002:00000ee8       ?szTitle@ShowMenuArgs@OleThread@@3PB_WB 10013ee8     OleThread.obj
 0002:00000eec       ?bAtCursorPos@ShowMenuArgs@OleThread@@3_NA 10013eec     OleThread.obj
 0002:00000ef0       ?nSelItem@ShowMenuArgs@OleThread@@3HA 10013ef0     OleThread.obj
 0002:00000ef4       ?Menu@ShowMenuArgs@OleThread@@3PAVCFarMenu@@A 10013ef4     OleThread.obj
 0002:00000ef8       ?nItem@OpenPluginArgs@OleThread@@3HA 10013ef8     OleThread.obj
 0002:00000efc       ?enRes@OpenPluginArgs@OleThread@@3W4EDoMenu@CPlugin@@A 10013efc     OleThread.obj
 0002:00000f00       ?nOpenFrom@OpenPluginArgs@OleThread@@3HA 10013f00     OleThread.obj
 0002:00000f04       ?hTerminator@OleThread@@3PAVCThreadTerminator@1@A 10013f04     OleThread.obj
 0002:00000f08       ?hNeedInvoke@OleThread@@3PAVCHandle@@A 10013f08     OleThread.obj
 0002:00000f0c       ?hInvokeDone@OleThread@@3PAVCHandle@@A 10013f0c     OleThread.obj
 0002:00000f10       ?hStop@OleThread@@3PAVCHandle@@A 10013f10     OleThread.obj
 0002:00000f14       ?hShowMenu@OleThread@@3PAVCHandle@@A 10013f14     OleThread.obj
 0002:00000f18       ?hMenuDone@OleThread@@3PAVCHandle@@A 10013f18     OleThread.obj
 0002:00000f1c       ?hThread@OleThread@@3PAXA  10013f1c     OleThread.obj
 0002:0000173c       __aenvptr                  1001473c     LIBCMT:dllcrt0.obj
 0002:00001740       __wenvptr                  10014740     LIBCMT:dllcrt0.obj
 0002:00001744       ___error_mode              10014744     LIBCMT:dllcrt0.obj
 0002:00001748       ___app_type                10014748     LIBCMT:dllcrt0.obj
 0002:0000174c       ?_pnhHeap@@3P6AHI@ZA       1001474c     LIBCMT:handler.obj
 0002:000017d8       _gpFlsAlloc                100147d8     LIBCMT:tidtable.obj
 0002:000017dc       _gpFlsGetValue             100147dc     LIBCMT:tidtable.obj
 0002:000017e0       _gpFlsSetValue             100147e0     LIBCMT:tidtable.obj
 0002:000017e4       _gpFlsFree                 100147e4     LIBCMT:tidtable.obj
 0002:000017e8       __maxwait                  100147e8     LIBCMT:crtheap.obj
 0002:000017ec       __umaskval                 100147ec     LIBCMT:crt0dat.obj
 0002:000017f0       ___argc                    100147f0     LIBCMT:crt0dat.obj
 0002:000017f4       ___argv                    100147f4     LIBCMT:crt0dat.obj
 0002:000017f8       ___wargv                   100147f8     LIBCMT:crt0dat.obj
 0002:000017fc       __environ                  100147fc     LIBCMT:crt0dat.obj
 0002:00001800       ___initenv                 10014800     LIBCMT:crt0dat.obj
 0002:00001804       __wenviron                 10014804     LIBCMT:crt0dat.obj
 0002:00001808       ___winitenv                10014808     LIBCMT:crt0dat.obj
 0002:0000180c       __pgmptr                   1001480c     LIBCMT:crt0dat.obj
 0002:00001810       __wpgmptr                  10014810     LIBCMT:crt0dat.obj
 0002:00001814       __exitflag                 10014814     LIBCMT:crt0dat.obj
 0002:00001818       __C_Termination_Done       10014818     LIBCMT:crt0dat.obj
 0002:0000181c       __C_Exit_Done              1001481c     LIBCMT:crt0dat.obj
 0002:00001928       __crtheap                  10014928     LIBCMT:heapinit.obj
 0002:00001f60       __newmode                  10014f60     LIBCMT:_newmode.obj
 0002:000020bc       ___mbulinfo                100150bc     LIBCMT:mbctype.obj
 0002:000020c8       ___mbcodepage              100150c8     LIBCMT:mbctype.obj
 0002:000020cc       ___ismbcodepage            100150cc     LIBCMT:mbctype.obj
 0002:000020d0       ___mblcid                  100150d0     LIBCMT:mbctype.obj
 0002:000020d4       ?__pInconsistency@@3P6AXXZA 100150d4     LIBCMT:hooks.obj
 0002:000020f0       ___pPurecall               100150f0     LIBCMT:inithelp.obj
 0002:000020f4       ___pInvalidArgHandler      100150f4     LIBCMT:invarg.obj
 0002:0000210c       ?pArgList@UnDecorator@@0PAVReplicator@@A 1001510c     LIBCMT:undname.obj
 0002:00002110       ?pZNameList@UnDecorator@@0PAVReplicator@@A 10015110     LIBCMT:undname.obj
 0002:00002114       ?pTemplateArgList@UnDecorator@@0PAVReplicator@@A 10015114     LIBCMT:undname.obj
 0002:00002118       ?gName@UnDecorator@@0PBDB  10015118     LIBCMT:undname.obj
 0002:0000211c       ?name@UnDecorator@@0PBDB   1001511c     LIBCMT:undname.obj
 0002:00002120       ?outputString@UnDecorator@@0PADA 10015120     LIBCMT:undname.obj
 0002:00002124       ?maxStringLength@UnDecorator@@0HA 10015124     LIBCMT:undname.obj
 0002:00002128       ?disableFlags@UnDecorator@@0KA 10015128     LIBCMT:undname.obj
 0002:0000212c       ?m_pGetParameter@UnDecorator@@0P6APADJ@ZA 1001512c     LIBCMT:undname.obj
 0002:00002130       ?fExplicitTemplateParams@UnDecorator@@0_NA 10015130     LIBCMT:undname.obj
 0002:00002131       ?fGetTemplateArgumentList@UnDecorator@@0_NA 10015131     LIBCMT:undname.obj
 0002:0000246c       ___lconv_static_null       1001546c     LIBCMT:lconv.obj
 0002:00002470       ___lconv_static_W_null     10015470     LIBCMT:lconv.obj
 0002:00002474       ___locale_changed          10015474     LIBCMT:setlocal.obj
 0002:00002478       ___fastflag                10015478     LIBCMT:_fpinit_.obj
 0002:0000247c       __outputformat             1001547c     LIBCMT:outputformat.obj
 0002:00002480       __debugger_hook_dummy      10015480     <common>
 0002:00002484       __nhandle                  10015484     <common>
 0002:000024a0       ___pioinfo                 100154a0     <common>
 0002:000025a0       ___env_initialized         100155a0     <common>
 0002:000025a4       ___onexitend               100155a4     <common>
 0002:000025a8       ___onexitbegin             100155a8     <common>
 0002:000025ac       ___mbctype_initialized     100155ac     <common>
 0002:000025b0       ___dyn_tls_init_callback   100155b0     <common>
 0002:000025b4       __pDestructExceptionObject 100155b4     <common>
 0002:000025b8       ___sse2_available          100155b8     <common>
 0002:000025bc       __acmdln                   100155bc     <common>

 entry point at        0001:00008afb

 Static symbols

 0001:00008a05       ___DllMainCRTStartup       10009a05 f   LIBCMT:dllcrt0.obj
 0001:00008c63       __onexit_nolock            10009c63 f   LIBCMT:onexit.obj
 0001:00009120       __unwind_handler           1000a120 f   LIBCMT:exsup.obj
 0001:00009240       _ValidateScopeTableHandlers 1000a240 f   LIBCMT:eh3valid.obj
 0001:00009d4a       _doexit                    1000ad4a f   LIBCMT:crt0dat.obj
 0001:0000a241       _parse_cmdline             1000b241 f   LIBCMT:stdargv.obj
 0001:0000b474       ?CPtoLCID@@YAHH@Z          1000c474 f   LIBCMT:mbctype.obj
 0001:0000b4a3       ?setSBCS@@YAXPAUthreadmbcinfostruct@@@Z 1000c4a3 f   LIBCMT:mbctype.obj
 0001:0000b507       ?setSBUpLow@@YAXPAUthreadmbcinfostruct@@@Z 1000c507 f   LIBCMT:mbctype.obj
 0001:0000b7c2       ?getSystemCP@@YAHH@Z       1000c7c2 f   LIBCMT:mbctype.obj
 0001:0000bd76       _siglookup                 1000cd76 f   LIBCMT:winsig.obj
 0001:0000c138       ?x_ismbbtype_l@@YAHPAUlocaleinfo_struct@@IHH@Z 1000d138 f   LIBCMT:ismbbyte.obj
 0001:0000c240       __unwind_handler4          1000d240 f   LIBCMT:exsup4.obj
 0001:0000cc71       ?__crtLCMapStringA_stat@@YAHPAUlocaleinfo_struct@@KKPBDHPADHHH@Z 1000dc71 f   LIBCMT:a_map.obj
 0001:0000ce9e       ?__crtGetStringTypeA_stat@@YAHPAUlocaleinfo_struct@@KPBDHPAGHHH@Z 1000de9e f   LIBCMT:a_str.obj
 0001:0000d75f       __shift                    1000e75f f   LIBCMT:cvt.obj
 0001:0000d7a4       __cftoe2_l                 1000e7a4 f   LIBCMT:cvt.obj
 0001:0000dd62       __cftof2_l                 1000ed62 f   LIBCMT:cvt.obj
 0001:000100b4       __hw_cw                    100110b4 f   LIBCMT:_ieee87_.obj
 0001:00010142       ___hw_cw_sse2              10011142 f   LIBCMT:_ieee87_.obj
 0001:0001074a       ??__Fnomem@?5???2@YAPAXI@Z@YAXXZ 1001174a f   LIBCMT:new.obj
